:020000040000FA
:04080000F1EF0BF019
:1008100003B276EF05F0F2B494EF05F09EB09CEFD2
:1008200005F09EB2A4EF05F0F2A81AEF04F0F2B2C0
:1008300025EF04F0F2A620EF04F0F2B022EF04F06E
:10084000A0EF0BF0F296F290FF00CD90F2929EA0F6
:100850002FEF04F00101533F2FEF04F0542BAEC1F2
:10086000B2F1AFC1B3F1B0C1B4F1B1C1B5F1AAC138
:10087000AEF1ABC1AFF1ACC1B0F1ADC1B1F1A6C148
:10088000AAF1A7C1ABF1A8C1ACF1A9C1ADF1A2C158
:10089000A6F1A3C1A7F1A4C1A8F1A5C1A9F19EC168
:1008A000A2F19FC1A3F1A0C1A4F1A1C1A5F19AC178
:1008B0009EF19BC19FF19CC1A0F19DC1A1F196C188
:1008C0009AF197C19BF198C19CF199C19DF1CECF4E
:1008D00096F1CFCF97F153C198F154C199F1CF6AF6
:1008E000CE6A0101536B546B9E90CD800FBC0F8E6E
:1008F0000FBA7EEF04F00F8AA0EF0BF00F8C0FBE43
:10090000BAEF04F096C19AF197C19BF198C19CF19E
:1009100099C19DF19AC19EF19BC19FF19CC1A0F12B
:100920009DC1A1F19EC1A2F19FC1A3F1A0C1A4F1FB
:10093000A1C1A5F1A2C1A6F1A3C1A7F1A4C1A8F1CB
:10094000A5C1A9F1A6C1AAF1A7C1ABF1A8C1ACF19B
:10095000A9C1ADF1AAC1AEF1ABC1AFF1ACC1B0F16B
:10096000ADC1B1F1AEC1B2F1AFC1B3F1B0C1B4F13B
:10097000B1C1B5F101015E6B5F6B606B616B96514C
:100980005E2797515F2398516023995161239A51B3
:100990005E279B515F239C5160239D5161239E5193
:1009A0005E279F515F23A0516023A1516123A25173
:1009B0005E27A3515F23A4516023A5516123A65153
:1009C0005E27A7515F23A8516023A9516123AA5133
:1009D0005E27AB515F23AC516023AD516123AE5113
:1009E0005E27AF515F23B0516023B1516123B251F3
:1009F0005E27B3515F23B4516023B5516123D89072
:100A00000101613360335F335E33D890010161339C
:100A100060335F335E33D8900101613360335F33FD
:100A20005E3300C10CF101C10DF102C10EF103C131
:100A30000FF104C110F105C111F106C112F107C196
:100A400013F108C114F109C115F10AC116F10BC166
:100A500017F134C135F111B839EF05F00101620E1B
:100A6000046F010E056F000E066F000E076F42EF58
:100A700005F00101A70E046F020E056F000E066F50
:100A8000000E076F5EC100F15FC101F160C102F1AC
:100A900061C103F16EEC36F003BF04D019BE02D081
:100AA00019A0108C11A05AEF05F010BA5AEF05F0FA
:100AB0000F80108A0CC100F10DC101F10EC102F1CD
:100AC0000FC103F110C104F111C105F112C106F10A
:100AD00013C107F114C108F115C109F116C10AF1DA
:100AE00017C10BF135C134F1A0EF0BF00392ABB29B
:100AF000AB98AB88030103EE00F080517F0BE92631
:100B000004C0EFFF802B8151805D700BD8A48B82D5
:100B100000008051815D700BD8A48B9281518019A7
:100B2000D8B40790A0EF0BF0F2940101453FA0EF7D
:100B30000BF0462BA0EF0BF09E900101533FA0EF6E
:100B40000BF0542BA0EF0BF09E9211B873EF08F04E
:100B5000040066A1ACEF05F08BB4B6EF05F010AC65
:100B6000B6EF05F08B84109CB7EF05F08B9407B4BB
:100B700009EF06F007B009EF06F01EC620F61FC603
:100B800021F61CC61EF61DC61FF61AC61CF61BC68D
:100B90001DF606C608F607C609F604C606F605C61B
:100BA00007F602C604F603C605F626C628F627C6CB
:100BB00029F624C626F625C627F622C624F623C61D
:100BC00025F60EC610F60FC611F60CC60EF60DC6AB
:100BD0000FF60AC60CF60BC60DF62EC630F62FC65B
:100BE00031F62CC62EF62DC62FF62AC62CF62BC6AD
:100BF0002DF616C618F617C619F614C616F615C63B
:100C000017F612C614F613C615F64FEC38F0FDECC5
:100C100037F0077C07AC24EF06F0C274C2B41EEFB5
:100C200006F0C3CFB7F5C4CFB8F50501D890B833F7
:100C3000B733D890B833B73325EF06F0C3CF55F1AB
:100C4000C4CF56F125EF06F0C28207B492EF06F04A
:100C500047C14BF148C14CF149C14DF14AC14EF178
:100C60005EC162F15FC163F160C164F161C165F1B0
:100C700096C1B6F197C1B7F198C1B8F199C1B9F170
:100C80009AC1BAF19BC1BBF19CC1BCF19DC1BDF140
:100C90009EC1BEF19FC1BFF1A0C1C0F1A1C1C1F110
:100CA000A2C1C2F1A3C1C3F1A4C1C4F1A5C1C5F1E0
:100CB000A6C1C6F1A7C1C7F1A8C1C8F1A9C1C9F1B0
:100CC000AAC1CAF1ABC1CBF1ACC1CCF1ADC1CDF180
:100CD000AEC1CEF1AFC1CFF1B0C1D0F1B1C1D1F150
:100CE000B2C1D2F1B3C1D3F1B4C1D4F1B5C1D5F120
:100CF000B7C5B9F5B8C5BAF5B9C5BBF5BAC5BCF540
:100D0000010155515B2756515C23E86A5D230E2E85
:100D100092EF06F05CC157F15DC158F15B6B5C6B03
:100D20005D6B078E0201002FA0EF0BF03C0E006FF1
:100D30001A50E00BE00AE866128818BE02D018B418
:100D4000108E00C10CF101C10DF102C10EF103C101
:100D50000FF104C110F105C111F106C112F107C173
:100D600013F108C114F109C115F10AC116F10BC143
:100D700017F134C135F105012F51000AD8B46CEFD9
:100D800007F005012F51010AD8B4F6EF06F005016E
:100D90002F51020AD8B437EF07F005012F51030A8B
:100DA000D8B437EF07F005012F51040AD8B437EF54
:100DB00007F005012F51050AD8B437EF07F00501F8
:100DC0002F51060AD8B437EF07F005012F51070A53
:100DD000D8B437EF07F005012F51320AD8B4F4EF39
:100DE00006F02F6B6CEF07F06CEF07F0050157670B
:100DF00001EF07F0586701EF07F0596701EF07F0BF
:100E00005A6705EF07F06CEF07F05BC500F15CC5B2
:100E100001F15DC502F15EC503F10101010E046F30
:100E2000000E056F000E066F000E076F6EEC36F0B9
:100E300000C15BF501C15CF502C15DF503C15EF562
:100E400000672AEF07F001672AEF07F002672AEF31
:100E500007F003676CEF07F057C55BF558C55CF505
:100E600059C55DF55AC55EF50F886CEF07F00501B1
:100E700030673DEF07F06CEF07F00FBE52EF07F061
:100E800010A057EF07F0010147674EEF07F04867E2
:100E90004EEF07F049674EEF07F04A6752EF07F051
:100EA00057EF07F007AE57EF07F069EF07F00501BE
:100EB000312F6CEF07F03C0E316F302F6CEF07F0E5
:100EC0000101000E626FE00E636FA50E646F010EEC
:100ED000656F0501306B0F880501666B37B772EFE0
:100EE00007F066810CC100F10DC101F10EC102F1E4
:100EF0000FC103F110C104F111C105F112C106F1D6
:100F000013C107F114C108F115C109F116C10AF1A5
:100F100017C10BF135C134F100C10CF101C10DF164
:100F200002C10EF103C10FF104C110F105C111F1AD
:100F300006C112F107C113F108C114F109C115F17D
:100F40000AC116F10BC117F134C135F101018A67ED
:100F5000B1EF07F08B67B1EF07F08C67B1EF07F0E7
:100F60008D67B5EF07F0E5EF07F08EC100F18FC197
:100F700001F190C102F191C103F10101010E046F71
:100F8000000E056F000E066F000E076F6EEC36F058
:100F900000C18EF101C18FF102C190F103C191F145
:100FA0000067DAEF07F00167DAEF07F00267DAEFC0
:100FB00007F00367E5EF07F08AC18EF18BC18FF16F
:100FC0008CC190F18DC191F10F80D57ED5BE6DD0D1
:100FD000D6CF47F1D7CF48F145C149F1E86AE8CF0C
:100FE0004AF119BE02D019A0108C109047C100F12F
:100FF00048C101F149C102F14AC103F101010A0EE0
:10100000046F000E056F000E066F000E076F6EEC8A
:1010100036F003AF1080010154A71BEF08F00F9AC0
:101020000F9C0F9E0101000E5E6F600E5F6F3D0E04
:10103000606F080E616F010147BF2BEF08F0486732
:101040002BEF08F049672BEF08F04A672BEF08F009
:10105000F28850EF08F0F2985E6B5F6B606B616B2B
:10106000966B976B986B996B9A6B9B6B9C6B9D6B5C
:101070009E6B9F6BA06BA16BA26BA36BA46BA56B0C
:10108000A66BA76BA86BA96BAA6BAB6BAC6BAD6BBC
:10109000AE6BAF6BB06BB16BB26BB36BB46BB56B6C
:1010A000D76AD66A0101456B466B0CC100F10DC1D0
:1010B00001F10EC102F10FC103F110C104F111C120
:1010C00005F112C106F113C107F114C108F115C1F0
:1010D00009F116C10AF117C10BF135C134F1A0EFC6
:1010E0000BF0A0EF0BF00201002FB7EF0AF0D59E36
:1010F000D6CF47F1D7CF48F145C149F1E86AE8CFEB
:101100004AF1D76AD66A0101456B466BD58E1A50F3
:10111000E00BE00AE866128818BE02D018B4108E00
:1011200017AE1C8C00C10CF101C10DF102C10EF112
:1011300003C10FF104C110F105C111F106C112F193
:1011400007C113F108C114F109C115F10AC116F163
:101150000BC117F134C135F10FA0109A11B8BCEFD3
:1011600008F00101620E046F010E056F000E066F9C
:10117000000E076FC5EF08F00101A70E046F020E05
:10118000056F000E066F000E076F47C100F148C1E2
:1011900001F149C102F14AC103F16EEC36F003BF1F
:1011A000D8EF08F019BE02D019A0108C11B00F8032
:1011B0000CC100F10DC101F10EC102F10FC103F12B
:1011C00010C104F111C105F112C106F113C107F1FB
:1011D00014C108F115C109F116C10AF117C10BF1CB
:1011E00035C134F102013C0E006F00C10CF101C1A8
:1011F0000DF102C10EF103C10FF104C110F105C1DF
:1012000011F106C112F107C113F108C114F109C1AE
:1012100015F10AC116F10BC117F134C135F1050101
:101220002F51000AD8B4C0EF09F005012F51010A6F
:10123000D8B44AEF09F005012F51020AD8B48BEF58
:1012400009F005012F51030AD8B48BEF09F005010D
:101250002F51040AD8B48BEF09F005012F51050A6C
:10126000D8B48BEF09F005012F51060AD8B48BEFE3
:1012700009F005012F51070AD8B48BEF09F00501D9
:101280002F51320AD8B448EF09F02F6BC0EF09F0A4
:10129000C0EF09F00501576755EF09F0586755EFA2
:1012A00009F0596755EF09F05A6759EF09F0C0EF97
:1012B00009F05BC500F15CC501F15DC502F15EC5D9
:1012C00003F10101010E046F000E056F000E066FA1
:1012D000000E076F6EEC36F000C15BF501C15CF5E6
:1012E00002C15DF503C15EF500677EEF09F001679D
:1012F0007EEF09F002677EEF09F00367C0EF09F0A7
:1013000057C55BF558C55CF559C55DF55AC55EF521
:101310000F88C0EF09F00501306791EF09F0C0EFC9
:1013200009F00FBEA6EF09F010A0ABEF09F0010124
:101330004767A2EF09F04867A2EF09F04967A2EFFB
:1013400009F04A67A6EF09F0ABEF09F007AEABEF83
:1013500009F0BDEF09F00501312FC0EF09F03C0E97
:10136000316F302FC0EF09F00101000E626FE00E07
:10137000636FA50E646F010E656F0501306B0F88FA
:101380000501666B37B7C6EF09F066810CC100F145
:101390000DC101F10EC102F10FC103F110C104F141
:1013A00011C105F112C106F113C107F114C108F111
:1013B00015C109F116C10AF117C10BF135C134F19C
:1013C00000C10CF101C10DF102C10EF103C10FF119
:1013D00004C110F105C111F106C112F107C113F1E9
:1013E00008C114F109C115F10AC116F10BC117F1B9
:1013F00034C135F101018A6705EF0AF08B6705EF0B
:101400000AF08C6705EF0AF08D6709EF0AF039EFF3
:101410000AF08EC100F18FC101F190C102F191C1BA
:1014200003F10101010E046F000E056F000E066F3F
:10143000000E076F6EEC36F000C18EF101C18FF126
:1014400002C190F103C191F100672EEF0AF001672C
:101450002EEF0AF002672EEF0AF0036739EF0AF069
:101460008AC18EF18BC18FF18CC190F18DC191F148
:101470000F80109047C100F148C101F149C102F14C
:101480004AC103F101010A0E046F000E056F000E40
:10149000066F000E076F6EEC36F003AF108001018F
:1014A00054A75FEF0AF00F9A0F9C0F9E0101000EE8
:1014B0005E6F600E5F6F3D0E606F080E616F47C11B
:1014C00000F148C101F149C102F14AC103F1010132
:1014D000140E046F050E056F000E066F000E076FE9
:1014E0006EEC36F003AF78EF0AF0F2889DEF0AF069
:1014F000F2985E6B5F6B606B616B966B976B986B32
:10150000996B9A6B9B6B9C6B9D6B9E6B9F6BA06B9F
:10151000A16BA26BA36BA46BA56BA66BA76BA86B4F
:10152000A96BAA6BAB6BAC6BAD6BAE6BAF6BB06BFF
:10153000B16BB26BB36BB46BB56B0CC100F10DC189
:1015400001F10EC102F10FC103F110C104F111C18B
:1015500005F112C106F113C107F114C108F115C15B
:1015600009F116C10AF117C10BF135C134F10400BC
:101570008BB4C2EF0AF010ACC2EF0AF08B84109C5F
:10158000C3EF0AF08B9407B415EF0BF007B015EF1B
:101590000BF01EC620F61FC621F61CC61EF61DC681
:1015A0001FF61AC61CF61BC61DF606C608F607C6A9
:1015B00009F604C606F605C607F602C604F603C613
:1015C00005F626C628F627C629F624C626F625C619
:1015D00027F622C624F623C625F60EC610F60FC639
:1015E00011F60CC60EF60DC60FF60AC60CF60BC6A3
:1015F0000DF62EC630F62FC631F62CC62EF62DC6A9
:101600002FF62AC62CF62BC62DF616C618F617C6C8
:1016100019F614C616F615C617F612C614F613C632
:1016200015F64FEC38F0FDEC37F0077C07AC30EFE7
:101630000BF0C274C2B42AEF0BF0C3CFB7F5C4CF1E
:10164000B8F50501D890B833B733D890B833B7336D
:1016500031EF0BF0C3CF55F1C4CF56F131EF0BF0A2
:10166000C28207B49EEF0BF047C14BF148C14CF169
:1016700049C14DF14AC14EF15EC162F15FC163F1F2
:1016800060C164F161C165F196C1B6F197C1B7F16E
:1016900098C1B8F199C1B9F19AC1BAF19BC1BBF136
:1016A0009CC1BCF19DC1BDF19EC1BEF19FC1BFF106
:1016B000A0C1C0F1A1C1C1F1A2C1C2F1A3C1C3F1D6
:1016C000A4C1C4F1A5C1C5F1A6C1C6F1A7C1C7F1A6
:1016D000A8C1C8F1A9C1C9F1AAC1CAF1ABC1CBF176
:1016E000ACC1CCF1ADC1CDF1AEC1CEF1AFC1CFF146
:1016F000B0C1D0F1B1C1D1F1B2C1D2F1B3C1D3F116
:10170000B4C1D4F1B5C1D5F1B7C5B9F5B8C5BAF50D
:10171000B9C5BBF5BAC5BCF5010155515B2756519A
:101720005C23E86A5D230E2E9EEF0BF05CC157F13F
:101730005DC158F15B6B5C6B5D6B078EA0EF0BF0CE
:1017400002C0E0FF005001C0D8FF1000A6B2A6EF13
:101750000BF00CC0A9FF0BC0A8FFA69EA69CA684F8
:10176000F29E550EA76EAA0EA76EA682F28EA694C2
:10177000A6B2B8EF0BF00C2A1200A96EA69EA69C8A
:10178000A680A8500C2A120004012C0E826F48EC8F
:101790000FF069EC37F00C50BDEC0BF0E8CF00F126
:1017A0000C50BDEC0BF0E8CF01F101AFDDEF0BF019
:1017B0000101FF0E026FFF0E036F0CEC37F029677B
:1017C000E9EF0BF00401200E826F48EC0FF0EEEF12
:1017D0000BF004012D0E826F48EC0FF036EC35F063
:1017E0001200076A0F6A106A116A126A136A0F01FF
:1017F0000D0EC16E860EC06E030EC26E0F01680E16
:10180000896E130E926E080E8A6E8A6AF30E936EBC
:101810008B6A900E946EC80EBDEC0BF0E8CFE8FF1B
:101820001098E8A0108810A805D00E0E226E8E0E1B
:10183000236E04D00F0E226E8F0E236E07EC39F04C
:10184000F18EF19EFC0EBDEC0BF0E8CF0BF00BA07F
:1018500011800BA211820BA411840BA81188C90E50
:10186000BDEC0BF0E8CF17F0CA0EBDEC0BF0E8CFE3
:1018700018F0CB0EBDEC0BF0E8CF19F0CC0EBDECA0
:101880000BF0E8CF1AF0CD0EBDEC0BF0E8CF2FF047
:101890001C6A1D6A0E6A01015B6B5C6B5D6B576BAA
:1018A000586BF29A0101476B486B496B4A6B4B6B63
:1018B0004C6B4D6B4E6B4F6B506B516B526B456B62
:1018C000466BD76AD66A0F01280ED56EF28A9D90B4
:1018D000B00ECD6E01015E6B5F6B606B616B626B16
:1018E000636B646B656B666B676B686B696B536B83
:1018F000546BCF6ACE6A0F9A0F9C0F9E9D80760E16
:10190000CA6E9D8202013C0E006FCC6A160EBDECC1
:101910000BF0E8CF00F1170EBDEC0BF0E8CF01F1B2
:10192000180EBDEC0BF0E8CF02F1190EBDEC0BF078
:10193000E8CF03F1010103AFB8EF0CF069EC37F029
:10194000160E0C6E00C10BF0A6EC0BF0170E0C6E11
:1019500001C10BF0A6EC0BF0180E0C6E02C10BF0DF
:10196000A6EC0BF0190E0C6E03C10BF0A6EC0BF0FD
:1019700000C18AF101C18BF102C18CF103C18DF16B
:1019800000C18EF101C18FF102C190F103C191F14B
:101990001A0EBDEC0BF0E8CF00F11B0EBDEC0BF006
:1019A000E8CF01F11C0EBDEC0BF0E8CF02F11D0EEB
:1019B000BDEC0BF0E8CF03F1010103AF0EEF0DF02A
:1019C00069EC37F01A0E0C6E00C10BF0A6EC0BF0B0
:1019D0001B0E0C6E01C10BF0A6EC0BF01C0E0C6E76
:1019E00002C10BF0A6EC0BF01D0E0C6E03C10BF048
:1019F000A6EC0BF01A0EBDEC0BF0E8CF00F11B0EBD
:101A0000BDEC0BF0E8CF01F11C0EBDEC0BF0E8CF04
:101A100002F11D0EBDEC0BF0E8CF03F100C192F115
:101A200001C193F102C194F103C195F1240EAC6E92
:101A3000900EAB6E240EAC6E080EB86E000EB06E3B
:101A40001F0EAF6E0401806B816B0F01900EAB6EA9
:101A50000F019D8A0301806B816BC26B8B928FECAF
:101A60003DF08FEC3DF0880EBDEC0BF0E8CF00F1BF
:101A7000890EBDEC0BF0E8CF01F1010101AF59EF88
:101A80000DF069EC37F0880E0C6E00C10BF0A6EC7F
:101A90000BF0890E0C6E01C10BF0A6EC0BF0880E5A
:101AA000BDEC0BF0E8CF00F1890EBDEC0BF0E8CFF8
:101AB00001F100C140F601C141F602C142F603C185
:101AC00043F6E7EC40F06EEC3BF0200EBDEC0BF083
:101AD000E8CF2FF505012F51FF0AD8A477EF0DF0BD
:101AE0002F6B200E0C6E2FC50BF0A6EC0BF0050132
:101AF000010E306F3C0E316F250EBDEC0BF0E8CFC0
:101B000000F1260EBDEC0BF0E8CF01F1270EBDEC85
:101B10000BF0E8CF02F1280EBDEC0BF0E8CF03F19B
:101B2000010103AFAEEF0DF069EC37F0250E0C6E3E
:101B300000C10BF0A6EC0BF0260E0C6E01C10BF0F1
:101B4000A6EC0BF0270E0C6E02C10BF0A6EC0BF00E
:101B5000280E0C6E03C10BF0A6EC0BF000C157F57C
:101B600001C158F502C159F503C15AF500C15BF531
:101B700001C15CF502C15DF503C15EF5290EBDEC46
:101B80000BF0E8CF5FF5050160515F5DD8A05FC540
:101B900060F505012F51020A0EE181B8DBEF0DF06F
:101BA0000501602FD8EF0DF05FC560F5DBEF0DF09C
:101BB00081BA26EF41F0210EBDEC0BF0E8CF00F129
:101BC000220EBDEC0BF0E8CF01F1230EBDEC0BF0C3
:101BD000E8CF02F1240EBDEC0BF0E8CF03F10101D8
:101BE00003AF21EF0EF069EC37F0210E0C6E00C14F
:101BF0000BF0A6EC0BF0220E0C6E01C10BF0A6EC64
:101C00000BF0230E0C6E02C10BF0A6EC0BF0240EB1
:101C10000C6E03C10BF0A6EC0BF0210EBDEC0BF02B
:101C2000E8CF00F1220EBDEC0BF0E8CF01F1230E5E
:101C3000BDEC0BF0E8CF02F1240EBDEC0BF0E8CFC9
:101C400003F100C161F501C162F502C163F503C191
:101C500064F5B6EC3AF0B8EC39F010EC39F0050167
:101C60002F51030A12E005012F51040A1DE005015E
:101C70002F51050A24E005012F51060A32E0050123
:101C80002F51070A38E084EF0EF0B0C500F10101D2
:101C90000F0E001701010051000A36E0010100514A
:101CA000050A32E081EF0EF0B0C500F101010F0E20
:101CB000001701010051000A27E081EF0EF0050135
:101CC000B051000A21E00501B051150A1DE00501DF
:101CD000B051300A19E00501B051450A15E081EF15
:101CE0000EF00501B051000A0FE00501B051300AB5
:101CF0000BE081EF0EF00501B051000A05E081EF25
:101D00000EF081BA26EF41F0A1EC38F00790000107
:101D1000F28EF28C12AE03D012BC5BEF20F007B053
:101D2000CBEF32F00FB067EF2CF010BE67EF2CF066
:101D300012B867EF2CF00FB804EF26F003018051C2
:101D400081197F0BD8B4CBEF32F013EE00F0815144
:101D50007F0BE126812BE7CFE8FFE00BD8B4CBEF78
:101D600032F023EE82F0C2513F0BD926E7CFDFFFDE
:101D7000C22BDF50780AD8A4CBEF32F007808EC197
:101D800000F18FC101F190C102F191C103F1010194
:101D9000040E046F000E056F000E066F000E076F35
:101DA0006EEC36F000AFDEEF0EF00101030E8E6F29
:101DB000000E8F6F000E906F000E916F0301825125
:101DC000720AD8B44CEF2CF08251520AD8B44CEFBE
:101DD0002CF08251750AD8B44CEF2CF08251630A72
:101DE000D8B485EF2FF08251690AD8B4FBEF28F000
:101DF00082517A0AD8B40EEF2AF08251490AD8B437
:101E00009AEF28F08251500AD8B4B8EF27F08251E7
:101E1000700AD8B4FBEF27F08251540AD8B426EFE9
:101E200028F08251740AD8B46CEF28F08251410A2C
:101E3000D8B45EEF10F082514B0AD8B45CEF0FF0CB
:101E400082516D0AD8B491EF14F082514D0AD8B482
:101E5000AAEF14F08251730AD8B47CEF2BF08251B0
:101E6000530AD8B4E1EF2BF082514C0AD8B40DEFED
:101E70001CF08251760AD8B439EF15F08251590A14
:101E8000D8B4E2EF13F012AE01D0128CBCEF2FF0F9
:101E9000040114EE00F080517F0BE12682C4E7FFBD
:101EA000802B120004010D0E826F48EC0FF00A0E19
:101EB000826F48EC0FF0120004014B0E826F48EC69
:101EC0000FF004012C0E826F48EC0FF081B802D0A5
:101ED0002FB630D003018351430AD8B4A1EF0FF0DD
:101EE00003018351630AD8B4A3EF0FF003018351B8
:101EF000520AD8B4A5EF0FF003018351720AD8B487
:101F0000A7EF0FF003018351470AD8B4A9EF0FF0F0
:101F100003018351670AD8B4ABEF0FF0030183517B
:101F2000540AD8B4ADEF0FF003018351740AD8B44A
:101F30001CEF10F003018351550AD8B4AFEF0FF036
:101F400082D02F807AD02F9078D02F8276D02F9287
:101F500074D02F8472D02F9470D02F866ED084C30B
:101F600030F185C331F186C332F187C333F101010A
:101F7000296BB7EC37F02EEC37F000C104F101C14A
:101F800005F102C106F103C107F1AAEC37F0200EFA
:101F9000F86EF76AF66A0900F5CF2CF10900F5CF63
:101FA0002DF10900F5CF2EF10900F5CF2FF1090031
:101FB000F5CF30F10900F5CF31F10900F5CF32F15D
:101FC0000900F5CF33F10101296BB7EC37F02EECA6
:101FD00037F06EEC36F00067F5EF0FF00167F5EFC4
:101FE0000FF00267F5EF0FF0036701D025D0040171
:101FF0004E0E826F48EC0FF004016F0E826F48ECBA
:102000000FF004014D0E826F48EC0FF00401610ED9
:10201000826F48EC0FF00401740E826F48EC0FF0F1
:102020000401630E826F48EC0FF00401680E826FAA
:1020300048EC0FF0BAEF2FF02F96CD0E0C6E2FC09C
:102040000BF0A6EC0BF0CD0EBDEC0BF0E8CF2FF0B3
:102050002FB006D00401630E826F48EC0FF005D05C
:102060000401430E826F48EC0FF02FB206D004013A
:10207000720E826F48EC0FF005D00401520E826F91
:1020800048EC0FF02FB406D00401670E826F48ECC5
:102090000FF005D00401470E826F48EC0FF02FB609
:1020A00006D00401740E826F48EC0FF005D00401D5
:1020B000540E826F48EC0FF0BAEF2FF00401410E7E
:1020C000826F48EC0FF003018351310AD8B402EF5C
:1020D00013F003018351320AD8B432EF12F0030136
:1020E0008351330AD8B4BBEF11F003018351340A92
:1020F000D8B4ABEF10F003018351350AD8B488EFA0
:1021000010F004013F0E826F48EC0FF0BAEF2FF091
:1021100004012C0E826F48EC0FF003018451300A49
:10212000D8B49BEF10F003018451310AD8B4A3EF67
:1021300010F0F4EF11F08B900401300E826F48EC38
:102140000FF0A9EF10F08B800401310E826F48EC84
:102150000FF0BAEF2FF0CC0EBDEC0BF0E8CF0BF088
:1021600004012C0E826F48EC0FF003018451310AF8
:10217000D8B4CFEF10F003018451300AD8B4D1EFB6
:1021800010F0030184514D0AD8B4DBEF10F00301C5
:102190008451540AD8B4E2EF10F0F9EF10F08A84B9
:1021A00001D08A940BAE04D00BAC02D00BBA21D074
:1021B000E00E0B1218D01F0E0B168539E844E00B09
:1021C0000B1211D0E00E0B16AAEC37F085C332F1DA
:1021D00086C333F10101296BB7EC37F02EEC37F0F1
:1021E00000511F0B0B12CC0E0C6E0BC00BF0A6ECAB
:1021F0000BF00401340E826F48EC0FF004012C0E3A
:10220000826F48EC0FF0CC0EBDEC0BF0E8CF1AF06B
:102210008AB406D00401300E826F48EC0FF005D06E
:102220000401310E826F48EC0FF004012C0E826F16
:1022300048EC0FF01A38E840070BE8CF82F40401AD
:10224000300E822748EC0FF004012C0E826F48EC10
:102250000FF069EC37F01A501F0BE8CF00F10CECCF
:1022600037F032C182F40401300E822748EC0FF0BF
:1022700033C182F40401300E822748EC0FF00401D0
:102280002C0E826F48EC0FF069EC37F02DC000F196
:1022900000AF0BD0FF0E016FFF0E026FFF0E036F3A
:1022A00004012D0E826F48EC0FF00CEC37F031C1B9
:1022B00082F40401300E822748EC0FF032C182F420
:1022C0000401300E822748EC0FF033C182F4040180
:1022D000300E822748EC0FF004012C0E826F48EC80
:1022E0000FF069EC37F02CC000F10CEC37F031C185
:1022F00082F40401300E822748EC0FF032C182F4E0
:102300000401300E822748EC0FF033C182F404013F
:10231000300E822748EC0FF004012C0E826F48EC3F
:102320000FF069EC37F02EC000F100AF0BD0FF0EBC
:10233000016FFF0E026FFF0E036F04012D0E826FFF
:1023400048EC0FF00CEC37F031C182F40401300E90
:10235000822748EC0FF032C182F40401300E82274C
:1023600048EC0FF033C182F40401300E822748ECB0
:102370000FF0BAEF2FF0CB0EBDEC0BF0E8CF0BF067
:1023800004012C0E826F48EC0FF003018451450AC2
:10239000D8B4DFEF11F003018451440AD8B4E2EF5E
:1023A00011F003018451300AD8B4E5EF11F00301B4
:1023B0008451310AD8B4E9EF11F0F4EF11F00B9E1B
:1023C000EEEF11F00B8EEEEF11F0FC0E0B16EEEFB0
:1023D00011F0FC0E0B160B80EEEF11F0CB0E0C6E15
:1023E0000BC00BF0A6EC0BF00401330E826F48EC2F
:1023F0000FF004012C0E826F48EC0FF0CB0EBDECF9
:102400000BF0E8CF19F019BE0DEF12F00401450EE4
:10241000826F48EC0FF012EF12F00401440E826F4D
:1024200048EC0FF004012C0E826F48EC0FF0040111
:10243000300E826F48EC0FF004012C0E826F48ECD6
:102440000FF019B02BEF12F00401300E826F48EC40
:102450000FF030EF12F00401310E826F48EC0FF0F4
:10246000BAEF2FF0CA0EBDEC0BF0E8CF0BF0040171
:102470002C0E826F48EC0FF003018451450AD8B44A
:102480006EEF12F003018451440AD8B471EF12F0D8
:10249000030184514D0AD8B47AEF12F0030184513C
:1024A000410AD8B474EF12F003018451460AD8B43B
:1024B00077EF12F003018451560AD8B482EF12F07C
:1024C00003018451500AD8B48DEF12F003018451F6
:1024D000520AD8B490EF12F099EF12F00B9E93EFDE
:1024E00012F00B8E93EF12F00B9C93EF12F00B8C0B
:1024F00093EF12F0FC0E0B1685C3E8FF030B0B12D3
:1025000093EF12F0C70E0B1685C3E8FF070BE846E2
:10251000E846E8460B1293EF12F00B8493EF12F0AB
:102520000B9493EF12F0CA0E0C6E0BC00BF0A6ECDE
:102530000BF0CA0EBDEC0BF0E8CF18F00401320E20
:10254000826F48EC0FF004012C0E826F48EC0FF004
:1025500018BEB2EF12F00401450E826F48EC0FF086
:10256000B7EF12F00401440E826F48EC0FF0040143
:102570002C0E826F48EC0FF018C0E8FF030BE8CF79
:1025800082F40401300E822748EC0FF004012C0E77
:10259000826F48EC0FF018BCD5EF12F00401410E29
:1025A000826F48EC0FF0DAEF12F00401460E826FF2
:1025B00048EC0FF004012C0E826F48EC0FF018C0AD
:1025C000E8FF380BE842E842E842E8CF82F4040131
:1025D000300E822748EC0FF004012C0E826F48EC7D
:1025E0000FF018B4FBEF12F00401520E826F48ECAA
:1025F0000FF000EF13F00401500E826F48EC0FF063
:10260000BAEF2FF0C90EBDEC0BF0E8CF0BF00401D0
:102610002C0E826F48EC0FF003018451450AD8B4A8
:1026200020EF13F003018451440AD8B423EF13F0D0
:10263000030184514D0AD8B426EF13F034EF13F0A0
:102640000B9E2EEF13F00B8E2EEF13F0F80E0B16E1
:1026500085C3E8FF070B0B122EEF13F0C90E0C6EAB
:102660000BC00BF0A6EC0BF00401310E826F48ECAE
:102670000FF004012C0E826F48EC0FF0C90EBDEC78
:102680000BF0E8CF17F017BE06D00401450E826F9D
:1026900048EC0FF005D00401440E826F48EC0FF0B7
:1026A00004012C0E826F48EC0FF017C0E8FF070BF7
:1026B000E8CF82F40401300E822748EC0FF00401C9
:1026C0002C0E826F48EC0FF0078069EC37F028C0C1
:1026D000E8FF003B00430043030B0CEC37F033C131
:1026E00082F40401300E822748EC0FF004012C0E16
:1026F000826F48EC0FF069EC37F028C001F1019FC0
:10270000019D29C000F101010CEC37F02FC182F4CA
:102710000401300E822748EC0FF030C182F404012E
:10272000300E822748EC0FF031C182F40401300EE4
:10273000822748EC0FF032C182F40401300E822768
:1027400048EC0FF033C182F40401300E822748ECCC
:102750000FF004012C0E826F48EC0FF069EC37F09B
:102760002AC001F12BC000F1D89001330033D8907A
:102770000133003301010CEC37F02FC182F4040166
:10278000300E822748EC0FF030C182F40401300E85
:10279000822748EC0FF031C182F40401300E822709
:1027A00048EC0FF032C182F40401300E822748EC6D
:1027B0000FF033C182F40401300E822748EC0FF091
:1027C000BAEF2FF0FC0EBDEC0BF0E8CF0BF00301DD
:1027D0008351520AD8B419EF14F003018351720ADD
:1027E000D8B41CEF14F003018351500AD8B41FEF82
:1027F00014F003018351700AD8B422EF14F00301DE
:102800008351550AD8B425EF14F003018351750A9A
:10281000D8B428EF14F003018351430AD8B431EF40
:1028200014F003018351630AD8B434EF14F03DEF80
:1028300014F00B9037EF14F00B8037EF14F00B927D
:1028400037EF14F00B8237EF14F00B9437EF14F0DE
:102850000B8437EF14F00B9637EF14F00B8637EF3D
:1028600014F00B9837EF14F00B8837EF14F0FC0ED0
:102870000C6E0BC00BF0A6EC0BF00401590E826F2E
:1028800048EC0FF01190119211941198FC0EBDECD0
:102890000BF0E8CF0BF00BA011800BA211820BA460
:1028A00011840BA8118811A05DEF14F00401520EE1
:1028B000826F48EC0FF062EF14F00401720E826F29
:1028C00048EC0FF011A86CEF14F00401430E826F76
:1028D00048EC0FF071EF14F00401630E826F48ECC6
:1028E0000FF011A27BEF14F00401500E826F48EC40
:1028F0000FF080EF14F00401700E826F48EC0FF0BF
:1029000011A48AEF14F00401550E826F48EC0FF009
:102910008FEF14F00401750E826F48EC0FF0BAEFE0
:102920002FF004016D0E826F48EC0FF0030183510C
:10293000300AD8B4E9EF14F003018351310AD8B456
:10294000FCEF14F003018351320AD8B40FEF15F0F5
:10295000BCEF2FF004014D0E826F48EC0FF0AAEC93
:1029600037F084C331F185C332F186C333F10101FD
:10297000296BB7EC37F02EEC37F003018351300AA6
:10298000D8B4D1EF14F003018351310AD8B4D9EF90
:1029900014F003018351320AD8B4E1EF14F0BCEF14
:1029A0002FF0FD0E0C6E00C10BF0A6EC0BF0E9EF62
:1029B00014F0FE0E0C6E00C10BF0A6EC0BF0FCEF59
:1029C00014F0FF0E0C6E00C10BF0A6EC0BF00FEF35
:1029D00015F00401300E826F48EC0FF004012C0E4C
:1029E000826F48EC0FF069EC37F0FD0EBDEC0BF098
:1029F000E8CF00F120EF15F00401310E826F48ECB2
:102A00000FF004012C0E826F48EC0FF069EC37F0E8
:102A1000FE0EBDEC0BF0E8CF00F120EF15F0040145
:102A2000320E826F48EC0FF069EC37F004012C0E87
:102A3000826F48EC0FF0FF0EBDEC0BF0E8CF00F119
:102A40000CEC37F031C182F40401300E822748ECDF
:102A50000FF032C182F40401300E822748EC0FF0EF
:102A600033C182F40401300E822748EC0FF0BAEF34
:102A70002FF003018351300AD8B4DEEF16F00301C2
:102A80008351310AD8B415EF17F003018351320A8C
:102A9000D8B4CAEF18F003018351330AD8B47FEFDA
:102AA0001AF003018351340AD8B425EF1BF0030157
:102AB0008351730AD8B4C0EF15F003018351760A2D
:102AC000D8B4C2EF15F003018351740AD8B4ADEF46
:102AD00015F003018351540AD8B472EF15F0D8A44D
:102AE000BCEF2FF00401760E826F48EC0FF004016A
:102AF000540E826F48EC0FF007840001880E0C6EB4
:102B0000AAEC37F02981030184512D0AD8B48BEF48
:102B100015F00101299185C32FF186C330F187C3D8
:102B200031F188C332F189C333F1B7EC37F02EECC1
:102B300037F000C10BF0A6EC0BF001C10BF0A6ECD6
:102B40000BF0880EBDEC0BF0E8CF40F6890EBDEC23
:102B50000BF0E8CF41F6B8EF15F00401760E826F66
:102B600048EC0FF00401740E826F48EC0FF00784FC
:102B70000001880E0C6EC4EC0BF0079465EF26F094
:102B8000C0EC15F00401760E826F48EC0FF00401E2
:102B9000760E826F48EC0FF00784E6EC33F0040108
:102BA0002C0E826F48EC0FF00101036B026B3BC6E9
:102BB00001F13AC600F101AFE3EF15F00101FF0E9C
:102BC000026FFF0E036F0CEC37F02967EAEF15F088
:102BD000EFEF15F004012D0E826F48EC0FF02FC1BE
:102BE00082F40401300E822748EC0FF030C182F4E9
:102BF0000401300E822748EC0FF031C182F4040149
:102C0000300E822748EC0FF032C182F40401300EFE
:102C1000822748EC0FF033C182F40401300E822782
:102C200048EC0FF004012C0E826F48EC0FF001010C
:102C3000036B026B3DC601F13CC600F101AF26EF0C
:102C400016F00101FF0E026FFF0E036F0CEC37F060
:102C500029672DEF16F032EF16F004012D0E826F6A
:102C600048EC0FF02FC182F40401300E822748ECAB
:102C70000FF030C182F40401300E822748EC0FF0CF
:102C800031C182F40401300E822748EC0FF032C1CA
:102C900082F40401300E822748EC0FF033C182F435
:102CA0000401300E822748EC0FF004012C0E826FD5
:102CB00048EC0FF00101036B026B3FC601F13EC609
:102CC00000F101AF69EF16F00101FF0E026FFF0E78
:102CD000036F0CEC37F0296770EF16F075EF16F004
:102CE00004012D0E826F48EC0FF02FC182F4040115
:102CF000300E822748EC0FF030C182F40401300E10
:102D0000822748EC0FF031C182F40401300E822793
:102D100048EC0FF032C182F40401300E822748ECF7
:102D20000FF033C182F40401300E822748EC0FF01B
:102D300004012C0E826F48EC0FF00101036B026B53
:102D400037C601F136C600F101AFACEF16F0010154
:102D5000FF0E026FFF0E036F0CEC37F02967B3EF25
:102D600016F0B8EF16F004012D0E826F48EC0FF04C
:102D70002FC182F40401300E822748EC0FF030C1DD
:102D800082F40401300E822748EC0FF031C182F446
:102D90000401300E822748EC0FF032C182F40401A6
:102DA000300E822748EC0FF033C182F40401300E5C
:102DB000822748EC0FF0079465EF26F00401760EA9
:102DC000826F48EC0FF00401300E826F48EC0FF078
:102DD00004012C0E826F48EC0FF0D7EC37F069EC51
:102DE00037F000C600F101C601F10CEC37F030C13C
:102DF00082F40401300E822748EC0FF031C182F4D6
:102E00000401300E822748EC0FF032C182F4040135
:102E1000300E822748EC0FF033C182F40401300EEB
:102E2000822748EC0FF065EF26F00401760E826FE2
:102E300048EC0FF00401310E826F48EC0FF007846C
:102E40000101036B026B02C600F103C601F101AF81
:102E50002EEF17F0FF0E026FFF0E036F0101076BDD
:102E6000066B04C604F105C605F105AF3CEF17F08B
:102E7000FF0E066FFF0E076F73EC36F00101076B54
:102E8000066B06C604F107C605F105AF4CEF17F057
:102E9000FF0E066FFF0E076F73EC36F00101076B34
:102EA000066B08C604F109C605F105AF5CEF17F023
:102EB000FF0E066FFF0E076F73EC36F0D89001011E
:102EC0000333023301330033D8900101033302335B
:102ED0000133003304012C0E826F48EC0FF0010126
:102EE000036B026B01C101F100C100F101AF7EEF84
:102EF00017F00101FF0E026FFF0E036F0CEC37F0AD
:102F0000296785EF17F08AEF17F004012D0E826F05
:102F100048EC0FF02FC182F40401300E822748ECF8
:102F20000FF030C182F40401300E822748EC0FF01C
:102F300031C182F40401300E822748EC0FF032C117
:102F400082F40401300E822748EC0FF033C182F482
:102F50000401300E822748EC0FF00101036B026B75
:102F60000AC600F10BC601F101AFBBEF17F0FF0E6F
:102F7000026FFF0E036F0101076B066B0CC604F1B5
:102F80000DC605F105AFC9EF17F0FF0E066FFF0E76
:102F9000076F73EC36F00101076B066B0EC604F188
:102FA0000FC605F105AFD9EF17F0FF0E066FFF0E44
:102FB000076F73EC36F00101076B066B10C604F166
:102FC00011C605F105AFE9EF17F0FF0E066FFF0E12
:102FD000076F73EC36F0D8900101033302330133ED
:102FE0000033D8900101033302330133003304016D
:102FF0002C0E826F48EC0FF00101036B026B01C1D4
:1030000001F100C100F101AF0BEF18F00101FF0E5B
:10301000026FFF0E036F0CEC37F0296712EF18F008
:1030200017EF18F004012D0E826F48EC0FF02FC13E
:1030300082F40401300E822748EC0FF030C182F494
:103040000401300E822748EC0FF031C182F40401F4
:10305000300E822748EC0FF032C182F40401300EAA
:10306000822748EC0FF033C182F40401300E82272E
:1030700048EC0FF00101036B026B12C600F113C69E
:1030800001F101AF48EF18F0FF0E026FFF0E036F62
:103090000101076B066B14C604F115C605F105AFF7
:1030A00056EF18F0FF0E066FFF0E076F73EC36F049
:1030B0000101076B066B16C604F117C605F105AFD3
:1030C00066EF18F0FF0E066FFF0E076F73EC36F019
:1030D0000101076B066B18C604F119C605F105AFAF
:1030E00076EF18F0FF0E066FFF0E076F73EC36F0E9
:1030F000D89001010333023301330033D89001012A
:10310000033302330133003304012C0E826F48EC89
:103110000FF00101036B026B01C101F100C100F16D
:1031200001AF98EF18F00101FF0E026FFF0E036F61
:103130000CEC37F029679FEF18F0A4EF18F00401AA
:103140002D0E826F48EC0FF02FC182F40401300E77
:10315000822748EC0FF030C182F40401300E822740
:1031600048EC0FF031C182F40401300E822748ECA4
:103170000FF032C182F40401300E822748EC0FF0C8
:1031800033C182F40401300E822748EC0FF007941B
:1031900065EF26F00401760E826F48EC0FF0040113
:1031A000320E826F48EC0FF007840101036B026B53
:1031B0001AC600F11BC601F101AFE3EF18F0FF0ED4
:1031C000026FFF0E036F0101076B066B1CC604F153
:1031D0001DC605F105AFF1EF18F0FF0E066FFF0EEB
:1031E000076F73EC36F00101076B066B1EC604F126
:1031F0001FC605F105AF01EF19F0FF0E066FFF0EB8
:10320000076F73EC36F00101076B066B20C604F103
:1032100021C605F105AF11EF19F0FF0E066FFF0E85
:10322000076F73EC36F0D89001010333023301339A
:103230000033D8900101033302330133003304011A
:103240002C0E826F48EC0FF00101036B026B01C181
:1032500001F100C100F101AF33EF19F00101FF0EE0
:10326000026FFF0E036F0CEC37F029673AEF19F08D
:103270003FEF19F004012D0E826F48EC0FF02FC1C3
:1032800082F40401300E822748EC0FF030C182F442
:103290000401300E822748EC0FF031C182F40401A2
:1032A000300E822748EC0FF032C182F40401300E58
:1032B000822748EC0FF033C182F40401300E8227DC
:1032C00048EC0FF00101036B026B22C600F123C62C
:1032D00001F101AF70EF19F0FF0E026FFF0E036FE7
:1032E0000101076B066B24C604F125C605F105AF85
:1032F0007EEF19F0FF0E066FFF0E076F73EC36F0CE
:103300000101076B066B26C604F127C605F105AF60
:103310008EEF19F0FF0E066FFF0E076F73EC36F09D
:103320000101076B066B28C604F129C605F105AF3C
:103330009EEF19F0FF0E066FFF0E076F73EC36F06D
:10334000D89001010333023301330033D8900101D7
:10335000033302330133003304012C0E826F48EC37
:103360000FF00101036B026B01C101F100C100F11B
:1033700001AFC0EF19F00101FF0E026FFF0E036FE6
:103380000CEC37F02967C7EF19F0CCEF19F0040106
:103390002D0E826F48EC0FF02FC182F40401300E25
:1033A000822748EC0FF030C182F40401300E8227EE
:1033B00048EC0FF031C182F40401300E822748EC52
:1033C0000FF032C182F40401300E822748EC0FF076
:1033D00033C182F40401300E822748EC0FF0010162
:1033E000036B026B2AC600F12BC601F101AFFDEFA2
:1033F00019F0FF0E026FFF0E036F0101076B066BE2
:103400002CC604F12DC605F105AF0BEF1AF0FF0E27
:10341000066FFF0E076F73EC36F00101076B066B4A
:103420002EC604F12FC605F105AF1BEF1AF0FF0EF3
:10343000066FFF0E076F73EC36F00101076B066B2A
:1034400030C604F131C605F105AF2BEF1AF0FF0EBF
:10345000066FFF0E076F73EC36F0D890010103334F
:10346000023301330033D8900101033302330133B7
:10347000003304012C0E826F48EC0FF00101036B46
:10348000026B01C101F100C100F101AF4DEF1AF073
:103490000101FF0E026FFF0E036F0CEC37F029677E
:1034A00054EF1AF059EF1AF004012D0E826F48EC18
:1034B0000FF02FC182F40401300E822748EC0FF088
:1034C00030C182F40401300E822748EC0FF031C184
:1034D00082F40401300E822748EC0FF032C182F4EE
:1034E0000401300E822748EC0FF033C182F404014E
:1034F000300E822748EC0FF0079465EF26F00401A8
:10350000760E826F48EC0FF00401330E826F48ECA8
:103510000FF004012C0E826F48EC0FF085C382F48B
:1035200048EC0FF0640E0D6E03018551320A02E182
:103530006A0E0D6E03018551330A02E1700E0D6EA5
:1035400003018551340A02E1760E0D6E03018551A7
:10355000350A02E17C0E0D6E03018551360A02E147
:10356000820E0D6E03018651780A65E00DC00CF0E5
:10357000AAEC37F02981030187512D0AD8B4C3EF93
:103580001AF00101299188C32FF189C330F18AC350
:1035900031F18BC332F18CC333F1B7EC37F02EEC41
:1035A00037F000C10BF0A6EC0BF001C10BF0A6EC5C
:1035B0000BF0AAEC37F0298103018E512D0AD8B403
:1035C000E4EF1AF0010129918FC32FF190C330F17C
:1035D00091C331F192C332F193C333F1B7EC37F0B9
:1035E0002EEC37F000C10BF0A6EC0BF001C10BF094
:1035F000A6EC0BF0AAEC37F02981030195512D0AB6
:10360000D8B405EF1BF00101299196C32FF197C3A0
:1036100030F198C331F199C332F19AC333F1B7EC69
:1036200037F02EEC37F000C10BF0A6EC0BF001C127
:103630000BF0A6EC0BF00DC00CF0C4EC0BF0C4ECDE
:103640000BF0C4EC0BF065EF26F00401760E826FF0
:1036500048EC0FF00401340E826F48EC0FF00301C8
:103660008451780AD8B4FDEF1BF03E0E0C6EAAEC24
:1036700037F02981030185512D0AD8B442EF1BF0A0
:103680000101299186C32FF187C330F188C331F13D
:1036900089C332F18AC333F1B7EC37F02EEC37F03F
:1036A00000C10BF0A6EC0BF001C10BF0A6EC0BF087
:1036B000AAEC37F0298103018C512D0AD8B463EFAD
:1036C0001BF0010129918DC32FF18EC330F18FC3FF
:1036D00031F190C332F191C333F1B7EC37F02EECF6
:1036E00037F000C10BF0A6EC0BF001C10BF0A6EC1B
:1036F0000BF0AAEC37F02981030193512D0AD8B4BD
:1037000084EF1BF00101299194C32FF195C330F18F
:1037100096C331F197C332F198C333F1B7EC37F068
:103720002EEC37F000C10BF0A6EC0BF001C10BF052
:10373000A6EC0BF0AAEC37F0298103019A512D0A6F
:10374000D8B4A5EF1BF0010129919BC32FF19CC3B5
:1037500030F19DC331F19EC332F19FC333F1B7EC19
:1037600037F02EEC37F000C10BF0A6EC0BF001C1E6
:103770000BF0A6EC0BF0AAEC37F029810301A15164
:103780002D0AD8B4C6EF1BF001012991A2C32FF175
:10379000A3C330F1A4C331F1A5C332F1A6C333F101
:1037A000B7EC37F02EEC37F000C10BF0A6EC0BF0C5
:1037B00001C10BF0A6EC0BF0AAEC37F02981030154
:1037C000A8512D0AD8B4E7EF1BF001012991A9C334
:1037D0002FF1AAC330F1ABC331F1ACC332F1ADC3A9
:1037E00033F1B7EC37F02EEC37F000C10BF0A6EC5C
:1037F0000BF001C10BF0A6EC0BF03E0E0C6EC4EC0E
:103800000BF0C4EC0BF0C4EC0BF0C4EC0BF0C4EC0C
:103810000BF0C4EC0BF065EF26F003018351300A86
:10382000D8B408EF21F003018351310AD8B435EF41
:1038300022F003018351320AD8B4A3EF22F003012E
:103840008351330AD8B4B3EF22F003018351340A11
:10385000D8B4C3EF22F003018351350AD8B409EF7D
:1038600026F003018351360AD8B437EF26F003015E
:103870008351370AD8B4E0EF1EF003018351380AB0
:10388000D8B47EEF1FF003018351460AD8B45DEF30
:1038900025F0030183514D0AD8B459EF1DF00301FF
:1038A00083516D0AD8B473EF1DF0030183515A0A96
:1038B000D8B4AFEF21F003018351490AD8B437EFF0
:1038C00027F003018351500AD8B469EF26F00301B1
:1038D0008351540AD8B4E2EF26F003018351630AFE
:1038E000D8B493EF1DF003018351430AD8B48BEF92
:1038F0001EF003018351730AD8B491EF1DF0030148
:103900008351610AD8B4A6EF1CF003018351650A04
:10391000D8B458EF21F003018351450AD8B466EFBB
:1039200021F003018351620AD8B474EF21F003013E
:103930008351420AD8B482EF21F003018351760A01
:10394000D8B490EF21F0D8A4BCEF2FF004014C0EB6
:10395000826F48EC0FF00401610E826F48EC0FF0AB
:10396000B8EC39F004012C0E826F48EC0FF069ECD2
:1039700037F0AFC500F101010CEC37F031C182F432
:103980000401300E822748EC0FF032C182F40401AA
:10399000300E822748EC0FF033C182F40401300E60
:1039A000822748EC0FF004012C0E826F48EC0FF0D8
:1039B00069EC37F0B0C500F101010CEC37F031C112
:1039C00082F40401300E822748EC0FF032C182F4F9
:1039D0000401300E822748EC0FF033C182F4040159
:1039E000300E822748EC0FF004012C0E826F48EC59
:1039F0000FF069EC37F0B1C500F101010CEC37F0C4
:103A000031C182F40401300E822748EC0FF032C13C
:103A100082F40401300E822748EC0FF033C182F4A7
:103A20000401300E822748EC0FF004012C0E826F47
:103A300048EC0FF069EC37F0B2C500F101010CEC75
:103A400037F031C182F40401300E822748EC0FF0C8
:103A500032C182F40401300E822748EC0FF033C1EA
:103A600082F40401300E822748EC0FF004012C0E82
:103A7000826F48EC0FF069EC37F0B6C500F1010138
:103A80000CEC37F031C182F40401300E822748EC8F
:103A90000FF032C182F40401300E822748EC0FF09F
:103AA00033C182F40401300E822748EC0FF065EF39
:103AB00026F0AAEC37F084C333F1B7EC37F02EECE4
:103AC00037F0200E0C6E00C10BF0A6EC0BF000C11D
:103AD0002FF505012F51000A06E005012F51010ABB
:103AE00002E052EC3AF004014C0E826F48EC0FF009
:103AF00004014D0E826F48EC0FF004012C0E826F12
:103B000048EC0FF069EC37F02FC500F10CEC37F002
:103B100033C182F40401300E822748EC0FF065EFC8
:103B200026F026EF41F004014C0E826F48EC0FF0B6
:103B30000401630E826F48EC0FF010EC39F00401C1
:103B40002C0E826F48EC0FF0A8EC1DF065EF26F00C
:103B500069EC37F0B5C500F10101003B0F0E00170D
:103B60000CEC37F033C182F40401300E822748ECAC
:103B70000FF0B5C500F101010F0E010100170CECAB
:103B800037F033C182F40401300E822748EC0FF085
:103B900004012D0E826F48EC0FF0B4C500F1010155
:103BA000003B0F0E00170CEC37F033C182F4040118
:103BB000300E822748EC0FF0B4C500F101010F0E62
:103BC000010100170CEC37F033C182F40401300E10
:103BD000822748EC0FF004012D0E826F48EC0FF0A5
:103BE000B3C500F10101003B0F0E00170CEC37F0DC
:103BF00033C182F40401300E822748EC0FF0B3C5C4
:103C000000F101010F0E010100170CEC37F033C178
:103C100082F40401300E822748EC0FF00401200EDC
:103C2000826F48EC0FF0B2C500F10F0E01010017D2
:103C30000CEC37F033C182F40401300E822748ECDB
:103C40000FF00401200E826F48EC0FF0B1C500F1B7
:103C500001010101003B0F0E00170CEC37F033C1DE
:103C600082F40401300E822748EC0FF0B1C500F158
:103C700001010F0E010100170CEC37F033C182F483
:103C80000401300E822748EC0FF004013A0E826FD7
:103C900048EC0FF0B0C500F10101003B0F0E00171A
:103CA0000CEC37F033C182F40401300E822748EC6B
:103CB0000FF0B0C500F101010F0E010100170CEC6F
:103CC00037F033C182F40401300E822748EC0FF044
:103CD00004013A0E826F48EC0FF0AFC500F101010C
:103CE000003B0F0E00170CEC37F033C182F40401D7
:103CF000300E822748EC0FF0AFC500F101010F0E26
:103D000000170CEC37F033C182F40401300E822727
:103D100048EC0FF0120084C3E8FF0F0BE83AE8CF3D
:103D2000B5F585C3E8FF0F0B0501B51387C3E8FFA1
:103D30000F0BE83AE8CFB4F588C3E8FF0F0B050195
:103D4000B4138AC3E8FF0F0BE83AE8CFB3F58BC38F
:103D5000E8FF0F0B0501B3138DC3E8FF0F0BE8CF8E
:103D6000B2F58FC3E8FF0F0BE83AE8CFB1F590C387
:103D7000E8FF0F0B0501B11392C3E8FF0F0BE83A00
:103D8000E8CFB0F593C3E8FF0F0B0501B01395C35F
:103D9000E8FF0F0BE83AE8CFAFF596C3E8FF0F0B4B
:103DA0000501AF136BEC39F004014C0E826F48EC47
:103DB0000FF00401430E826F48EC0FF09DEF1DF0F1
:103DC000078404014C0E826F48EC0FF00401370E9B
:103DD000826F48EC0FF004012C0E826F48EC0FF05C
:103DE00005012E51130A06E005012E51170A0DE0B8
:103DF0007BEF1FF00101000E006F000E016F100E2F
:103E0000026F000E036F0EEF1FF00101000E006F36
:103E1000000E016F000E026F010E036F0CEC37F005
:103E20002AC182F40401300E822748EC0FF02BC126
:103E300082F40401300E822748EC0FF02CC182F48A
:103E40000401300E822748EC0FF02DC182F40401EA
:103E5000300E822748EC0FF02EC182F40401300EA0
:103E6000822748EC0FF02FC182F40401300E822724
:103E700048EC0FF030C182F40401300E822748EC88
:103E80000FF031C182F40401300E822748EC0FF0AC
:103E900032C182F40401300E822748EC0FF033C1A6
:103EA00082F40401300E822748EC0FF004012C0E3E
:103EB000826F48EC0FF00101200E006F000E016FC1
:103EC000000E026F000E036F0CEC37F031C182F46C
:103ED0000401300E822748EC0FF032C182F4040155
:103EE000300E822748EC0FF033C182F40401300E0B
:103EF000822748EC0FF0079465EF26F00501216B4F
:103F0000226B236B246B04014C0E826F48EC0FF084
:103F10000401380E826F48EC0FF004012C0E826F02
:103F200048EC0FF00101200E006F000E016F000E33
:103F3000026F000E036F0CEC37F02AC182F404010B
:103F4000300E822748EC0FF02BC182F40401300EB2
:103F5000822748EC0FF02CC182F40401300E822736
:103F600048EC0FF02DC182F40401300E822748EC9A
:103F70000FF02EC182F40401300E822748EC0FF0BE
:103F80002FC182F40401300E822748EC0FF030C1BB
:103F900082F40401300E822748EC0FF031C182F424
:103FA0000401300E822748EC0FF032C182F4040184
:103FB000300E822748EC0FF033C182F40401300E3A
:103FC000822748EC0FF004012C0E826F48EC0FF0B2
:103FD00025C500F126C501F127C502F128C503F169
:103FE0000101200E046F000E056F000E066F000E1B
:103FF000076F9FEC36F000C133F501C134F502C103
:1040000035F503C136F50CEC37F02AC182F4040112
:10401000300E822748EC0FF02BC182F40401300EE1
:10402000822748EC0FF02CC182F40401300E822765
:1040300048EC0FF02DC182F40401300E822748ECC9
:104040000FF02EC182F40401300E822748EC0FF0ED
:104050002FC182F40401300E822748EC0FF030C1EA
:1040600082F40401300E822748EC0FF031C182F453
:104070000401300E822748EC0FF032C182F40401B3
:10408000300E822748EC0FF033C182F40401300E69
:10409000822748EC0FF052EC0FF00501336758EF20
:1040A00020F0346758EF20F0356758EF20F036677E
:1040B00002D0F7EF20F0129E129C21C500F122C51C
:1040C00001F123C502F124C503F1899A400EC76EA0
:1040D000200EC66E9E96C69E0B0EC96EFF0E9EB635
:1040E00002D0E82EFCD79E96C69E02C1C9FFFF0EE5
:1040F0009EB602D0E82EFCD79E96C69E01C1C9FF8F
:10410000FF0E9EB602D0E82EFCD79E96C69E00C13A
:10411000C9FFFF0E9EB602D0E82EFCD79E96C69E23
:10412000C952FF0E9EB602D0E82EFCD70501200E24
:10413000326F040114EE00F080517F0BE1269E9651
:10414000C69EC952FF0E9EB602D0E82EFCD7C9CF3C
:10415000E7FF0401802B0501322F99EF20F0898AB7
:1041600033C500F134C501F135C502F136C503F19F
:104170000101010E046F000E056F000E066F000EA8
:10418000076F6EEC36F000C133F501C134F502C1A2
:1041900035F503C136F505013367D6EF20F03467F6
:1041A000D6EF20F03567D6EF20F0366702D0F7EF74
:1041B00020F021C500F122C501F123C502F124C57B
:1041C00003F10101200E046F000E056F000E066F53
:1041D000000E076F73EC36F000C121F501C122F526
:1041E00002C123F503C124F5128EBCEF2FF00401A8
:1041F000450E826F48EC0FF004014F0E826F48ECC1
:104200000FF00401460E826F48EC0FF065EF26F0C8
:104210000784E7EC40F069EC37F02DC500F10CECB9
:1042200037F004014C0E826F48EC0FF00401300EA1
:10423000826F48EC0FF004012C0E826F48EC0FF0F7
:1042400031C182F40401300E822748EC0FF032C1F4
:1042500082F40401300E822748EC0FF033C182F45F
:104260000401300E822748EC0FF004012C0E826FFF
:1042700048EC0FF069EC37F02EC500F10CEC37F08C
:1042800031C182F40401300E822748EC0FF032C1B4
:1042900082F40401300E822748EC0FF033C182F41F
:1042A0000401300E822748EC0FF0079465EF26F0EA
:1042B00004014C0E826F48EC0FF00401650E826F12
:1042C00048EC0FF012EC3BF065EF26F004014C0EC9
:1042D000826F48EC0FF00401450E826F48EC0FF03E
:1042E00029EC3BF065EF26F004014C0E826F48ECA0
:1042F0000FF00401620E826F48EC0FF057EC3BF0B8
:1043000065EF26F004014C0E826F48EC0FF00401BB
:10431000420E826F48EC0FF040EC3BF065EF26F068
:1043200004014C0E826F48EC0FF00401760E826F90
:1043300048EC0FF004012C0E826F48EC0FF010A82F
:1043400007D00401310E826F48EC0FF065EF26F0C4
:104350000401300E826F48EC0FF065EF26F0040187
:104360004C0E826F48EC0FF004015A0E826F48EC3D
:104370000FF004012C0E826F48EC0FF0E7EC40F0D8
:1043800069EC37F005012E51130A06E005012E51A4
:10439000170A0DE0E0EF21F00101000E006F000EA2
:1043A000016F100E026F000E036FE0EF21F00101AC
:1043B000000E006F000E016F000E026F010E036F02
:1043C0000101200E046F000E056F000E066F000E37
:1043D000076F9FEC36F00CEC37F02AC182F4040131
:1043E000300E822748EC0FF02BC182F40401300E0E
:1043F000822748EC0FF02CC182F40401300E822792
:1044000048EC0FF02DC182F40401300E822748ECF5
:104410000FF02EC182F40401300E822748EC0FF019
:104420002FC182F40401300E822748EC0FF030C116
:1044300082F40401300E822748EC0FF031C182F47F
:104440000401300E822748EC0FF032C182F40401DF
:10445000300E822748EC0FF033C182F40401300E95
:10446000822748EC0FF065EF26F0078404014C0E1C
:10447000826F48EC0FF00401310E826F48EC0FF0B0
:1044800004012C0E826F48EC0FF025C500F126C503
:1044900001F127C502F128C503F10101200E046FC7
:1044A000000E056F000E066F000E076F9FEC36F0D2
:1044B0000CEC37F02AC182F40401300E822748EC5C
:1044C0000FF02BC182F40401300E822748EC0FF06C
:1044D0002CC182F40401300E822748EC0FF02DC16C
:1044E00082F40401300E822748EC0FF02EC182F4D2
:1044F0000401300E822748EC0FF02FC182F4040132
:10450000300E822748EC0FF030C182F40401300EE7
:10451000822748EC0FF031C182F40401300E82276B
:1045200048EC0FF032C182F40401300E822748ECCF
:104530000FF033C182F40401300E822748EC0FF0F3
:10454000079465EF26F0078404014C0E826F48EC57
:104550000FF00401320E826F48EC0FF045EC3DF095
:10456000079465EF26F0078404014C0E826F48EC37
:104570000FF00401330E826F48EC0FF0A2EC3DF017
:10458000079440EF22F0078404014C0E826F48EC40
:104590000FF00401340E826F48EC0FF004012C0E72
:1045A000826F48EC0FF0AAEC37F084C32AF185C380
:1045B0002BF186C32CF187C32DF188C32EF189C35B
:1045C0002FF18AC330F18BC331F18CC332F18DC32B
:1045D00033F10101296BB7EC37F02EEC37F0200EE8
:1045E000046F000E056F000E066F000E076F7FEC64
:1045F00036F000C121F501C122F502C123F503C146
:1046000024F59AEC40F038C5AFF539C5B0F53AC598
:10461000B1F53BC5B2F53CC5B3F53DC5B4F53EC5F6
:10462000B5F5A8EC1DF004012C0E826F48EC0FF0DC
:104630003FC500F140C501F141C502F142C503F19A
:104640000101000E046F000E056F010E066F000ED3
:10465000076F9FEC36F00CEC37F0296732EF23F050
:1046600037EF23F004012D0E826F48EC0FF030C1BC
:1046700082F40401300E822748EC0FF031C182F43D
:104680000401300E822748EC0FF004012E0E826FD9
:1046900048EC0FF032C182F40401300E822748EC5E
:1046A0000FF033C182F40401300E822748EC0FF082
:1046B00004012C0E826F48EC0FF069EC37F043C513
:1046C00000F144C501F1E6EC30F004012C0E826FDC
:1046D00048EC0FF069EC37F045C500F10CEC37F011
:1046E00031C182F40401300E822748EC0FF032C150
:1046F00082F40401300E822748EC0FF033C182F4BB
:104700000401300E822748EC0FF004012C0E826F5A
:1047100048EC0FF00101036B026B4CC501F14BC576
:1047200000F101AF99EF23F00101FF0E026FFF0EC0
:10473000036F0CEC37F02967A0EF23F0A5EF23F00F
:1047400004012D0E826F48EC0FF02FC182F404019A
:10475000300E822748EC0FF030C182F40401300E95
:10476000822748EC0FF031C182F40401300E822719
:1047700048EC0FF032C182F40401300E822748EC7D
:104780000FF033C182F40401300E822748EC0FF0A1
:1047900004012C0E826F48EC0FF00101036B026BD9
:1047A0004EC501F14DC500F101AFDCEF23F0010171
:1047B000FF0E026FFF0E036F0CEC37F02967E3EF7B
:1047C00023F0E8EF23F004012D0E826F48EC0FF088
:1047D0002FC182F40401300E822748EC0FF030C163
:1047E00082F40401300E822748EC0FF031C182F4CC
:1047F0000401300E822748EC0FF032C182F404012C
:10480000300E822748EC0FF033C182F40401300EE1
:10481000822748EC0FF004012C0E826F48EC0FF059
:104820000101036B026B50C501F14FC500F101AFEF
:104830001FEF24F00101FF0E026FFF0E036F0CEC5F
:1048400037F0296726EF24F02BEF24F004012D0E1A
:10485000826F48EC0FF02FC182F40401300E8227E2
:1048600048EC0FF030C182F40401300E822748EC8E
:104870000FF031C182F40401300E822748EC0FF0B2
:1048800032C182F40401300E822748EC0FF033C1AC
:1048900082F40401300E822748EC0FF004012C0E44
:1048A000826F48EC0FF00101036B026B52C501F1FE
:1048B00051C500F101AF62EF24F00101FF0E026F5C
:1048C000FF0E036F0CEC37F0296769EF24F06EEFF1
:1048D00024F004012D0E826F48EC0FF02FC182F4FA
:1048E0000401300E822748EC0FF030C182F404013D
:1048F000300E822748EC0FF031C182F40401300EF3
:10490000822748EC0FF032C182F40401300E822776
:1049100048EC0FF033C182F40401300E822748ECDA
:104920000FF004012C0E826F48EC0FF00101036BB5
:10493000026B54C501F153C500F101AFA5EF24F09E
:104940000101FF0E026FFF0E036F0CEC37F02967B9
:10495000ACEF24F0B1EF24F004012D0E826F48EC8F
:104960000FF02FC182F40401300E822748EC0FF0C3
:1049700030C182F40401300E822748EC0FF031C1BF
:1049800082F40401300E822748EC0FF032C182F429
:104990000401300E822748EC0FF033C182F4040189
:1049A000300E822748EC0FF004012C0E826F48EC89
:1049B0000FF00101036B026B56C501F155C500F103
:1049C00001AFE8EF24F00101FF0E026FFF0E036F4D
:1049D0000CEC37F02967EFEF24F0F4EF24F004013A
:1049E0002D0E826F48EC0FF02FC182F40401300EBF
:1049F000822748EC0FF030C182F40401300E822788
:104A000048EC0FF031C182F40401300E822748ECEB
:104A10000FF032C182F40401300E822748EC0FF00F
:104A200033C182F40401300E822748EC0FF00401F8
:104A30002C0E826F48EC0FF00101036B026B4AC52C
:104A400001F149C500F101AF2BEF25F00101FF0E87
:104A5000026FFF0E036F0CEC37F0296732EF25F081
:104A600037EF25F004012D0E826F48EC0FF02FC1B7
:104A700082F40401300E822748EC0FF030C182F43A
:104A80000401300E822748EC0FF031C182F404019A
:104A9000300E822748EC0FF032C182F40401300E50
:104AA000822748EC0FF033C182F40401300E8227D4
:104AB00048EC0FF0079465EF26F0AAEC37F085C3B9
:104AC0002AF186C32BF187C32CF188C32DF189C34A
:104AD0002EF18AC32FF18BC330F18CC331F18DC31A
:104AE00032F18EC333F10101296BB7EC37F02EECB4
:104AF00037F00101010E046F000E056F000E066F06
:104B0000000E076F6EEC36F0100E046F000E056F8E
:104B1000000E066F000E076F7FEC36F000C129F51E
:104B200001C12AF502C12BF503C12CF5CCEC3CF0F8
:104B300004014C0E826F48EC0FF00401460E826FA8
:104B400048EC0FF004012C0E826F48EC0FF025C5E5
:104B500000F126C501F127C502F128C503F10101C5
:104B6000100E046F000E056F000E066F000E076F2B
:104B70009FEC36F00CEC37F02AC182F40401300EC1
:104B8000822748EC0FF02BC182F40401300E8227FB
:104B900048EC0FF02CC182F40401300E822748EC5F
:104BA0000FF02DC182F40401300E822748EC0FF083
:104BB0002EC182F40401300E822748EC0FF02FC181
:104BC00082F40401300E822748EC0FF030C182F4E9
:104BD0000401300E822748EC0FF031C182F4040149
:104BE000300E822748EC0FF032C182F40401300EFF
:104BF000822748EC0FF033C182F40401300E822783
:104C000048EC0FF065EF26F00F98A2EC3DF0BCEFFA
:104C10002FF004014C0E826F48EC0FF00401350EAA
:104C2000826F48EC0FF004012C0E826F48EC0FF0FD
:104C300069EC37F00784B9C500F107940CEC37F044
:104C400031C182F40401300E822748EC0FF032C1EA
:104C500082F40401300E822748EC0FF033C182F455
:104C60000401300E822748EC0FF065EF26F065EC6A
:104C70003DF069EC37F037C500F10CEC37F004017A
:104C80004C0E826F48EC0FF00401360E826F48EC38
:104C90000FF004012C0E826F48EC0FF031C182F44A
:104CA0000401300E822748EC0FF032C182F4040177
:104CB000300E822748EC0FF033C182F40401300E2D
:104CC000822748EC0FF065EF26F052EC0FF0BCEFB6
:104CD0002FF004014C0E826F48EC0FF00401500ECF
:104CE000826F48EC0FF004012C0E826F48EC0FF03D
:104CF00085C32AF186C32BF187C32CF188C32DF11C
:104D000089C32EF18AC32FF18BC330F18CC331F1EB
:104D10008DC332F18EC333F10101B7EC37F02EECC5
:104D200037F003018451530A0DE0030184514D0A09
:104D300038E00401780E826F48EC0FF052EC0FF06F
:104D4000BCEF2FF00401530E826F48EC0FF0250EDC
:104D50000C6E00C10BF0A6EC0BF0260E0C6E01C120
:104D60000BF0A6EC0BF0270E0C6E02C10BF0A6ECBC
:104D70000BF0280E0C6E03C10BF0A6EC0BF000C17B
:104D800057F501C158F502C159F503C15AF500C1E3
:104D90005BF501C15CF502C15DF503C15EF546EF4F
:104DA00027F004014D0E826F48EC0FF0290E0C6EB7
:104DB00000C10BF0A6EC0BF000C15FF500C160F57F
:104DC00046EF27F004014C0E826F48EC0FF004010F
:104DD000540E826F48EC0FF004012C0E826F48ECE9
:104DE0000FF084C32AF185C32BF186C32CF187C34E
:104DF0002DF188C32EF189C32FF18AC330F18BC303
:104E000031F18DC332F18EC333F10101B7EC37F0CC
:104E10002EEC37F00101000E046F000E056F010E3D
:104E2000066F000E076F7FEC36F0210E0C6E00C18E
:104E30000BF0A6EC0BF0220E0C6E01C10BF0A6ECF1
:104E40000BF0230E0C6E02C10BF0A6EC0BF0240E3F
:104E50000C6E03C10BF0A6EC0BF000C161F501C1B3
:104E600062F502C163F503C164F546EF27F0040162
:104E70004C0E826F48EC0FF00401490E826F48EC33
:104E80000FF004012C0E826F48EC0FF0250EBDECE4
:104E90000BF0E8CF00F1260EBDEC0BF0E8CF01F1EE
:104EA000270EBDEC0BF0E8CF02F1280EBDEC0BF0A5
:104EB000E8CF03F10CEC37F0EFEC34F00401730EA3
:104EC000826F48EC0FF004012C0E826F48EC0FF05B
:104ED00069EC37F0290EBDEC0BF0E8CF00F10CECDB
:104EE00037F0EFEC34F00401730E826F48EC0FF0F2
:104EF00004012C0E826F48EC0FF05BC500F15CC51D
:104F000001F15DC502F15EC503F10CEC37F0EFEC89
:104F100034F00401730E826F48EC0FF004012C0E84
:104F2000826F48EC0FF069EC37F060C500F10CECD3
:104F300037F0EFEC34F004016D0E826F48EC0FF0A7
:104F400004012C0E826F48EC0FF061C500F162C5C0
:104F500001F163C502F164C503F1D7EC2FF0040140
:104F60002C0E826F48EC0FF052EC0FF0BCEF2FF0DC
:104F700083C32AF184C32BF185C32CF186C32DF1A1
:104F800087C32EF188C32FF189C330F18AC331F171
:104F90008BC332F18CC333F10101B7EC37F02EEC47
:104FA00037F0160E0C6E00C10BF0A6EC0BF0170ECE
:104FB0000C6E01C10BF0A6EC0BF0180E0C6E02C1CA
:104FC0000BF0A6EC0BF0190E0C6E03C10BF0A6EC67
:104FD0000BF000C18AF101C18BF102C18CF103C158
:104FE0008DF100C18EF101C18FF102C190F103C1B9
:104FF00091F19AEF28F083C32AF184C32BF185C382
:105000002CF186C32DF187C32EF188C32FF189C3FC
:1050100030F18AC331F18BC332F18CC333F101011A
:10502000B7EC37F02EEC37F000C18AF101C18BF1FB
:1050300002C18CF103C18DF100C18EF101C18FF16C
:1050400002C190F103C191F19AEF28F083C32AF1D4
:1050500084C32BF185C32CF186C32DF187C32EF1B8
:1050600088C32FF189C330F18AC331F18CC332F187
:105070008DC333F10101B7EC37F02EEC37F00101AD
:10508000000E046F000E056F010E066F000E076F15
:105090007FEC36F01A0E0C6E00C10BF0A6EC0BF094
:1050A0001B0E0C6E01C10BF0A6EC0BF01C0E0C6E6F
:1050B00002C10BF0A6EC0BF01D0E0C6E03C10BF041
:1050C000A6EC0BF000C192F101C193F102C194F181
:1050D00003C195F19AEF28F083C32AF184C32BF121
:1050E00085C32CF186C32DF187C32EF188C32FF120
:1050F00089C330F18AC331F18CC332F18DC333F1EE
:105100000101B7EC37F02EEC37F00101000E046F0F
:10511000000E056F010E066F000E076F7FEC36F074
:1051200000C192F101C193F102C194F103C195F163
:105130009AEF28F0160EBDEC0BF0E8CF00F1170E39
:10514000BDEC0BF0E8CF01F1180EBDEC0BF0E8CF91
:1051500002F1190EBDEC0BF0E8CF03F10CEC37F0C7
:10516000EFEC34F00401730E826F48EC0FF0040191
:105170002C0E826F48EC0FF08AC100F18BC101F157
:105180008CC102F18DC103F10CEC37F0EFEC34F07F
:105190000401730E826F48EC0FF004012C0E826F35
:1051A00048EC0FF01A0EBDEC0BF0E8CF00F11B0E2F
:1051B000BDEC0BF0E8CF01F11C0EBDEC0BF0E8CF1D
:1051C00002F11D0EBDEC0BF0E8CF03F1D7EC2FF090
:1051D00004012C0E826F48EC0FF092C100F193C1D4
:1051E00001F194C102F195C103F1D7EC2FF052EC1B
:1051F0000FF0BCEF2FF00401690E826F48EC0FF046
:1052000004012C0E826F48EC0FF00101040E006FB8
:10521000000E016F000E026F000E036F0CEC37F0F2
:105220002CC182F40401300E822748EC0FF02DC10E
:1052300082F40401300E822748EC0FF02EC182F474
:105240000401300E822748EC0FF02FC182F40401D4
:10525000300E822748EC0FF030C182F40401300E8A
:10526000822748EC0FF031C182F40401300E82270E
:1052700048EC0FF032C182F40401300E822748EC72
:105280000FF033C182F40401300E822748EC0FF096
:1052900004012C0E826F48EC0FF001010B0E006F21
:1052A000000E016F000E026F000E036F0CEC37F062
:1052B0002CC182F40401300E822748EC0FF02DC17E
:1052C00082F40401300E822748EC0FF02EC182F4E4
:1052D0000401300E822748EC0FF02FC182F4040144
:1052E000300E822748EC0FF030C182F40401300EFA
:1052F000822748EC0FF031C182F40401300E82277E
:1053000048EC0FF032C182F40401300E822748ECE1
:105310000FF033C182F40401300E822748EC0FF005
:1053200004012C0E826F48EC0FF00101300E006F6B
:10533000000E016F000E026F000E036F0CEC37F0D1
:105340002CC182F40401300E822748EC0FF02DC1ED
:1053500082F40401300E822748EC0FF02EC182F453
:105360000401300E822748EC0FF02FC182F40401B3
:10537000300E822748EC0FF030C182F40401300E69
:10538000822748EC0FF031C182F40401300E8227ED
:1053900048EC0FF032C182F40401300E822748EC51
:1053A0000FF033C182F40401300E822748EC0FF075
:1053B00004012C0E826F48EC0FF0200EF86EF76A95
:1053C000F66A04010900F5CF82F448EC0FF00900F9
:1053D000F5CF82F448EC0FF00900F5CF82F448ECE9
:1053E0000FF00900F5CF82F448EC0FF00900F5CF7B
:1053F00082F448EC0FF00900F5CF82F448EC0FF08E
:105400000900F5CF82F448EC0FF00900F5CF82F4E3
:1054100048EC0FF052EC0FF0BCEF2FF08351630A11
:10542000D8A4BAEF2FF08451610AD8A4BAEF2FF0B4
:1054300085516C0AD8A4BAEF2FF08651410A3FE09B
:105440008651440A1BE08651420AD8B472EF2AF012
:105450008651350AD8B446EF31F08651360AD8B4B1
:105460009BEF31F08651370AD8B404EF32F0865101
:10547000380AD8B462EF32F0BAEF2FF00798079AE3
:1054800004017A0E826F48EC0FF00401780E826FEF
:1054900048EC0FF00401640E826F48EC0FF0040139
:1054A000550E826F48EC0FF05BEF2AF004014C0EB2
:1054B000826F48EC0FF052EC0FF0BCEF2FF0078832
:1054C000079A04017A0E826F48EC0FF00401410E36
:1054D000826F48EC0FF00401610E826F48EC0FF010
:1054E0004FEF2AF00798078A04017A0E826F48EC82
:1054F0000FF00401420E826F48EC0FF00401610EC0
:10550000826F48EC0FF04FEF2AF00101666790EFD1
:105510002AF0676790EF2AF0686790EF2AF06967D2
:1055200015D04F679BEF2AF050679BEF2AF0516729
:105530009BEF2AF052670AD00101000E006F000EA7
:10554000016F000E026F000E036F120011B80AD037
:105550000101620E046F010E056F000E066F000E52
:10556000076F09D00101A70E046F020E056F000E30
:10557000066F000E076F66C100F167C101F168C1D7
:1055800002F169C103F16EEC36F003BF38EF2BF086
:10559000119A119C0101000E046FA80E056F550EA3
:1055A000066F020E076F66C100F167C101F168C1A5
:1055B00002F169C103F166C186F167C187F168C173
:1055C00088F169C189F16EEC36F003BF0BD001019F
:1055D000000E866FA80E876F550E886F020E896FBA
:1055E000118A119C0E0EBDEC0BF0E8CF18F10F0ED6
:1055F000BDEC0BF0E8CF19F1100EBDEC0BF0E8CFCD
:105600001AF1110EBDEC0BF0E8CF1BF1B7EC35F041
:1056100086C104F187C105F188C106F189C107F18E
:105620006EEC36F007827BEC35F0B7EC35F0079284
:105630007BEC35F086C100F187C101F188C102F130
:1056400089C103F107927BEC35F0CC0E046FE00EBC
:10565000056F870E066F050E076F6EEC36F000C102
:1056600018F101C119F102C11AF103C11BF13BD0BC
:10567000119C119A0101800E006F1A0E016F060E27
:10568000026F000E036F4FC104F150C105F151C10B
:1056900006F152C107F16EEC36F003AF05D069ECAC
:1056A00037F0118C119A12000E0EBDEC0BF0E8CF02
:1056B00018F10F0EBDEC0BF0E8CF19F1100EBDEC98
:1056C0000BF0E8CF1AF1110EBDEC0BF0E8CF1BF197
:1056D0004FC100F150C101F151C102F152C103F1BA
:1056E00007827BEC35F018C100F119C101F11AC134
:1056F00002F11BC103F112000401730E826F48EC2A
:105700000FF004012C0E826F48EC0FF0078462C189
:1057100066F163C167F164C168F165C169F14BC1AC
:105720004FF14CC150F14DC151F14EC152F157C131
:1057300059F158C15AF10794A2EC2BF052EC0FF03A
:10574000BCEF2FF066C100F167C101F168C102F141
:1057500069C103F101010CEC37F0EFEC34F0040106
:10576000630E826F48EC0FF004012C0E826F48EC40
:105770000FF04FC100F150C101F151C102F152C10E
:1057800003F101010CEC37F0EFEC34F00401660E8C
:10579000826F48EC0FF004012C0E826F48EC0FF082
:1057A00069EC37F059C100F15AC101F101010CEC6B
:1057B00037F0EFEC34F00401740E826F48EC0FF018
:1057C000120010820401530E826F48EC0FF00401A6
:1057D0002C0E826F48EC0FF083C32AF184C32BF1A7
:1057E00085C32CF186C32DF187C32EF188C32FF119
:1057F00089C330F18AC331F18BC332F18CC333F1E9
:105800000101B7EC37F02EEC37F000C166F101C1B1
:1058100067F102C168F103C169F18EC32AF18FC338
:105820002BF190C32CF191C32DF192C32EF193C3B0
:105830002FF194C330F195C331F196C332F197C380
:1058400033F10101B7EC37F02EEC37F000C14FF126
:1058500001C150F102C151F103C152F1AAEC37F07C
:1058600099C32FF19AC330F19BC331F19CC332F13C
:105870009DC333F10101B7EC37F02EEC37F000C1D6
:1058800059F101C15AF1A2EC2BF004012C0E826FE8
:1058900048EC0FF05BEF2CF0118E19A002D019AE7E
:1058A000108C18BE02D018A4108E8251520A02E148
:1058B0000F8201D00F928251750A02E1108401D04B
:1058C00010948251550A02E1108601D0109611A061
:1058D00003D011A401D01084078410B2C9EF2CF0BA
:1058E00010A4B5EF2CF0B6C166F1B7C167F1B8C12D
:1058F00068F1B9C169F1BAC16AF1BBC16BF1BCC150
:105900006CF1BDC16DF1BEC16EF1BFC16FF1C0C11F
:1059100070F1C1C171F1C2C172F1C3C173F1C4C1EF
:1059200074F1C5C175F1C6C176F1C7C177F1C8C1BF
:1059300078F1C9C179F1CAC17AF1CBC17BF1CCC18F
:105940007CF1CDC17DF1CEC17EF1CFC17FF1D0C15F
:1059500080F1D1C181F1D2C182F1D3C183F1D4C12F
:1059600084F1D5C185F1BDEF2CF062C166F163C150
:1059700067F164C168F165C169F14BC14FF14CC178
:1059800050F14DC151F14EC152F157C159F158C1B9
:105990005AF107940FA0EBEF2CF001019267D8EFBA
:1059A0002CF09367D8EF2CF09467D8EF2CF0956724
:1059B000DCEF2CF0EBEF2CF085EC2AF092C104F137
:1059C00093C105F194C106F195C107F16EEC36F073
:1059D00003BF82EF2FF085EC2AF00101000E046F67
:1059E000000E056F010E066F000E076F9FEC36F07C
:1059F00011A02CD011A22AD00CEC37F0296701D0CD
:105A000007D004012D0E826F48EC0FF080EF2FF0CD
:105A100030C182F40401300E822748EC0FF031C10E
:105A200082F40401300E822748EC0FF032C182F478
:105A30000401300E822748EC0FF033C182F40401D8
:105A4000300E822748EC0FF080EF2FF012A8C5D05F
:105A500012981AC01BF01B3A1B42070E1B160001BE
:105A60001B50000AD8B4B9EF2DF000011B50010AF9
:105A7000D8B445EF2DF000011B50020AD8B443EF13
:105A80002DF0EBEF2DF0EBEF2DF069EC37F02AC0A5
:105A900001F12BC000F1D89001330033D8900133CD
:105AA00000330101630E046F000E056F000E066FD8
:105AB000000E076F9FEC36F0280E046F000E056F86
:105AC000000E066F000E076F6EEC36F000C12DF071
:105AD00069EC37F028C001F1019F019D29C000F158
:105AE0000101A40E046F000E056F000E066F000E7C
:105AF000076F9FEC36F000C12CF000C104F101C12A
:105B000005F102C106F103C107F1640E006F000E3A
:105B1000016F000E026F000E036F6EEC36F0050E83
:105B2000046F000E056F000E066F000E076F9FECEE
:105B300036F000C104F101C105F102C106F103C153
:105B400007F169EC37F02DC000F16EEC36F000C1C2
:105B50002EF02EC0E8FF050F2D5C03E78A84EBEFE3
:105B60002DF02EC0E8FF0A0F2D5C01E68A94EBEFC2
:105B70002DF000C124F101C125F102C126F103C1BC
:105B800027F169EC37F06FEC37F01A501F0BE8CFB4
:105B900000F10101640E046F000E056F000E066F28
:105BA000000E076F7FEC36F024C104F125C105F12A
:105BB00026C106F127C107F16EEC36F003BF02D013
:105BC0008A9401D08A8424C100F125C101F126C143
:105BD00002F127C103F182EF2FF000C124F101C1CE
:105BE00025F102C126F103C127F110AE4CD0109E61
:105BF00000C108F101C109F102C10AF103C10BF1B1
:105C00000CEC37F030C1D6F131C1D7F132C1D8F147
:105C100033C1D9F108C100F109C101F10AC102F192
:105C20000BC103F101016C0E046F070E056F000E2E
:105C3000066F000E076F6EEC36F003BF04D0010153
:105C4000550EDA6F1CD008C100F109C101F10AC17B
:105C500002F10BC103F10101A40E046F060E056FE2
:105C6000000E066F000E076F6EEC36F003BF04D017
:105C700001017F0EDA6F03D00101FF0EDA6F1C8E77
:105C800011AE82EF2FF024C100F125C101F126C130
:105C900002F127C103F110A455EF2EF00401750E97
:105CA000826F48EC0FF05AEF2EF00401720E826FF3
:105CB00048EC0FF004012C0E826F48EC0FF00CEC56
:105CC00037F0296769EF2EF00401200E826F6CEF28
:105CD0002EF004012D0E826F48EC0FF030C182F4DB
:105CE0000401300E822748EC0FF031C182F4040128
:105CF000300E822748EC0FF004012E0E826F48EC24
:105D00000FF032C182F40401300E822748EC0FF00C
:105D100033C182F40401300E822748EC0FF00401F5
:105D20006D0E826F48EC0FF004012C0E826F48EC70
:105D30000FF04FC100F150C101F151C102F152C148
:105D400003F101010CEC37F0EFEC34F00401480EE4
:105D5000826F48EC0FF004017A0E826F48EC0FF06E
:105D600004012C0E826F48EC0FF066C100F167C190
:105D700001F168C102F169C103F101010CEC37F0D6
:105D8000EFEC34F00401630E826F48EC0FF0040175
:105D90002C0E826F48EC0FF066C100F167C101F173
:105DA00068C102F169C103F101010A0E046F000E1E
:105DB000056F000E066F000E076F7FEC36F0000EC9
:105DC000046F120E056F000E066F000E076F9FEC3A
:105DD00036F00CEC37F02AC182F40401300E822731
:105DE00048EC0FF02BC182F40401300E822748ECFE
:105DF0000FF02CC182F40401300E822748EC0FF022
:105E00002DC182F40401300E822748EC0FF02EC120
:105E100082F40401300E822748EC0FF02FC182F487
:105E20000401300E822748EC0FF030C182F40401E7
:105E3000300E822748EC0FF004012E0E826F48ECE2
:105E40000FF031C182F40401300E822748EC0FF0CC
:105E500032C182F40401300E822748EC0FF033C1C6
:105E600082F40401300E822748EC0FF00401730E17
:105E7000826F48EC0FF004012C0E826F48EC0FF09B
:105E800069EC37F059C100F15AC101F1E6EC30F08C
:105E90000FB24EEF2FF00FA080EF2FF004012C0E69
:105EA000826F48EC0FF0200EF86EF76AF66A040174
:105EB0000900F5CF82F448EC0FF00900F5CF82F429
:105EC00048EC0FF00900F5CF82F448EC0FF0090020
:105ED000F5CF82F448EC0FF00900F5CF82F448ECDE
:105EE0000FF00900F5CF82F448EC0FF00900F5CF70
:105EF00082F448EC0FF00900F5CF82F448EC0FF083
:105F000052EC0FF00F90BCEF2FF00401630E826F84
:105F100048EC0FF004012C0E826F48EC0FF0C2EC3D
:105F20002FF004012C0E826F48EC0FF035EC30F0AE
:105F300004012C0E826F48EC0FF0B1EC30F004013C
:105F40002C0E826F48EC0FF00101F80E006FCD0EA1
:105F5000016F660E026F030E036FD7EC2FF0040182
:105F60002C0E826F48EC0FF0C7EC30F052EC0FF0C3
:105F7000BCEF2FF052EC0FF00301C26B07901092B0
:105F8000CBEF32F0D8900E0EBDEC0BF0E8CF00F165
:105F90000F0EBDEC0BF0E8CF01F1100EBDEC0BF0D5
:105FA000E8CF02F1110EBDEC0BF0E8CF03F10101D7
:105FB000000E046F000E056F010E066F000E076FD6
:105FC0009FEC36F00CEC37F02AC182F40401300E5D
:105FD000822748EC0FF02BC182F40401300E822797
:105FE00048EC0FF02CC182F40401300E822748ECFB
:105FF0000FF02DC182F40401300E822748EC0FF01F
:106000002EC182F40401300E822748EC0FF02FC11C
:1060100082F40401300E822748EC0FF030C182F484
:106020000401300E822748EC0FF031C182F40401E4
:10603000300E822748EC0FF004012E0E826F48ECE0
:106040000FF032C182F40401300E822748EC0FF0C9
:1060500033C182F40401300E822748EC0FF00401B2
:106060006D0E826F48EC0FF01200120EBDEC0BF0BB
:10607000E8CF00F1130EBDEC0BF0E8CF01F1140EE8
:10608000BDEC0BF0E8CF02F1150EBDEC0BF0E8CF44
:1060900003F101010A0E046F000E056F000E066F7A
:1060A000000E076F7FEC36F0000E046F120E056FC6
:1060B000000E066F000E076F9FEC36F00CEC37F009
:1060C0002AC182F40401300E822748EC0FF02BC164
:1060D00082F40401300E822748EC0FF02CC182F4C8
:1060E0000401300E822748EC0FF02DC182F4040128
:1060F000300E822748EC0FF02EC182F40401300EDE
:10610000822748EC0FF02FC182F40401300E822761
:1061100048EC0FF030C182F40401300E822748ECC5
:106120000FF004012E0E826F48EC0FF031C182F4A3
:106130000401300E822748EC0FF032C182F40401D2
:10614000300E822748EC0FF033C182F40401300E88
:10615000822748EC0FF00401730E826F48EC0FF0B9
:1061600012000A0EBDEC0BF0E8CF00F10B0EBDECF7
:106170000BF0E8CF01F10C0EBDEC0BF0E8CF02F113
:106180000D0EBDEC0BF0E8CF03F1E6EF30F0060E9C
:10619000BDEC0BF0E8CF00F1070EBDEC0BF0E8CF43
:1061A00001F1080EBDEC0BF0E8CF02F1090EBDECD9
:1061B0000BF0E8CF03F1E6EF30F0010169EC37F0C6
:1061C000078457C100F158C101F107940101E80E9D
:1061D000046F800E056F000E066F000E076F7FECD8
:1061E00036F0000E046F040E056F000E066F000EF1
:1061F000076F9FEC36F0880E046F130E056F000ECC
:10620000066F000E076F6EEC36F00A0E046F000E7C
:10621000056F000E066F000E076F9FEC36F00CEC5A
:1062200037F0010129671AEF31F00401200E826F67
:106230001DEF31F004012D0E826F48EC0FF030C1DC
:1062400082F40401300E822748EC0FF031C182F451
:106250000401300E822748EC0FF032C182F40401B1
:10626000300E822748EC0FF004012E0E826F48ECAE
:106270000FF033C182F40401300E822748EC0FF096
:106280000401430E826F48EC0FF0120087C32AF11D
:1062900088C32BF189C32CF18AC32DF18BC32EF156
:1062A0008CC32FF18DC330F18EC331F190C332F125
:1062B00091C333F10101296BB7EC37F02EEC37F0C5
:1062C0000101000E046F000E056F010E066F000E37
:1062D000076F7FEC36F00E0E0C6E00C10BF0A6ECD3
:1062E0000BF00F0E0C6E01C10BF0A6EC0BF0100EB4
:1062F0000C6E02C10BF0A6EC0BF0110E0C6E03C17C
:106300000BF0A6EC0BF004017A0E826F48EC0FF054
:1063100004012C0E826F48EC0FF00401350E826FE1
:1063200048EC0FF004012C0E826F48EC0FF0C2EC29
:106330002FF05BEF2AF087C32AF188C32BF189C3C2
:106340002CF18AC32DF18BC32EF18CC32FF18DC399
:1063500030F18EC331F190C332F191C333F10101B9
:10636000296BB7EC37F02EEC37F0880E046F130E64
:10637000056F000E066F000E076F73EC36F0000E0F
:10638000046F040E056F000E066F000E076F7FECA2
:1063900036F00101E80E046F800E056F000E066FE7
:1063A000000E076F9FEC36F00A0E0C6E00C10BF06A
:1063B000A6EC0BF00B0E0C6E01C10BF0A6EC0BF073
:1063C0000C0E0C6E02C10BF0A6EC0BF00D0E0C6E59
:1063D00003C10BF0A6EC0BF004017A0E826F48ECBF
:1063E0000FF004012C0E826F48EC0FF00401360E02
:1063F000826F48EC0FF004012C0E826F48EC0FF016
:10640000B1EC30F05BEF2AF087C32AF188C32BF19F
:1064100089C32CF18AC32DF18BC32EF18CC32FF1CC
:106420008DC330F18FC331F190C332F191C333F199
:106430000101B7EC37F02EEC37F0000E046F120EAE
:10644000056F000E066F000E076F7FEC36F001013E
:106450000A0E046F000E056F000E066F000E076F28
:106460009FEC36F0120E0C6E00C10BF0A6EC0BF098
:10647000130E0C6E01C10BF0A6EC0BF0140E0C6E9B
:1064800002C10BF0A6EC0BF0150E0C6E03C10BF065
:10649000A6EC0BF004017A0E826F48EC0FF00401B9
:1064A0002C0E826F48EC0FF00401370E826F48EC1F
:1064B0000FF004012C0E826F48EC0FF035EC30F039
:1064C0005BEF2AF087C32AF188C32BF189C32CF133
:1064D0008AC32DF18BC32EF18CC32FF18DC330F104
:1064E0008EC331F190C332F191C333F10101296BB5
:1064F000B7EC37F02EEC37F0880E046F130E056FF3
:10650000000E066F000E076F73EC36F0000E046F7E
:10651000040E056F000E066F000E076F7FEC36F05D
:106520000101E80E046F800E056F000E066F000E6D
:10653000076F9FEC36F0060E0C6E00C10BF0A6EC58
:106540000BF0070E0C6E01C10BF0A6EC0BF0080E61
:106550000C6E02C10BF0A6EC0BF0090E0C6E03C121
:106560000BF0A6EC0BF004017A0E826F48EC0FF0F2
:1065700004012C0E826F48EC0FF00401380E826F7C
:1065800048EC0FF004012C0E826F48EC0FF0C7ECC2
:1065900030F05BEF2AF007A83EEF33F00101800EE8
:1065A000006F1A0E016F060E026F000E036F4BC1D3
:1065B00004F14CC105F14DC106F14EC107F16EEC7D
:1065C00036F003BF84EF33F0E9EC34F04BC100F157
:1065D0004CC101F14DC102F14EC103F107827BECC8
:1065E00035F018C104F119C105F11AC106F11BC13A
:1065F00007F1F80E006FCD0E016F660E026F030EED
:10660000036F6EEC36F00E0E0C6E00C10BF0A6ECB4
:106610000BF00F0E0C6E01C10BF0A6EC0BF0100E80
:106620000C6E02C10BF0A6EC0BF0110E0C6E03C148
:106630000BF0A6EC0BF00784010169EC37F057C1B1
:1066400000F158C101F107940A0E0C6E00C10BF065
:10665000A6EC0BF00B0E0C6E01C10BF0A6EC0BF0D0
:106660000C0E0C6E02C10BF0A6EC0BF00D0E0C6EB6
:1066700003C10BF0A6EC0BF084EF33F007AA84EF14
:1066800033F00784010169EC37F057C100F158C1BC
:1066900001F10794060E0C6E00C10BF0A6EC0BF096
:1066A000070E0C6E01C10BF0A6EC0BF0080E0C6E81
:1066B00002C10BF0A6EC0BF0090E0C6E03C10BF03F
:1066C000A6EC0BF0078462C100F163C101F164C163
:1066D00002F165C103F10794120E0C6E00C10BF0BC
:1066E000A6EC0BF0130E0C6E01C10BF0A6EC0BF038
:1066F000140E0C6E02C10BF0A6EC0BF0150E0C6E16
:1067000003C10BF0A6EC0BF00798079A0401805127
:1067100081197F0B0DE09EA8FED714EE00F0815189
:106720007F0BE126E750812B0F01AD6E86EF33F032
:1067300005012F51010A13E081AAAFEF33F00501E3
:106740002F51000A0AE00FB8AFEF33F005013067B0
:10675000AFEF33F00FB8AFEF33F026EF41F081B871
:10676000C4EF33F0B8EC39F005012F51020A02E012
:10677000C4EF33F0602FC4EF33F05FC560F505015F
:10678000010E306F3C0E316F8AEF0EF00601325170
:10679000385D3351D8A0010F395D800BD8A4D5EFF7
:1067A00033F032C638F633C639F6120006013251DC
:1067B000365D3351D8A0010F375D800BD8B4E5EFBB
:1067C00033F032C636F633C637F6120007841AC6DF
:1067D00032F61BC633F61CC638F61DC639F6C6ECB3
:1067E00033F01EC632F61FC633F6C6EC33F020C6B1
:1067F00032F621C633F6C6EC33F01AC632F61BC6A3
:1068000033F61CC636F61DC637F6D6EC33F01EC678
:1068100032F61FC633F6D6EC33F020C632F621C668
:1068200033F6D6EC33F03851365F3951D8A03929D8
:10683000375F69EC37F036C600F137C601F175EC09
:1068400037F000C13AF601C13BF622C632F623C644
:1068500033F624C638F625C639F6C6EC33F026C61C
:1068600032F627C633F6C6EC33F028C632F629C610
:1068700033F6C6EC33F022C632F623C633F624C60E
:1068800036F625C637F6D6EC33F026C632F627C6DE
:1068900033F6D6EC33F028C632F629C633F6D6ECFA
:1068A00033F03851365F3951D8A03929375F69EC58
:1068B00037F036C600F137C601F175EC37F000C18C
:1068C0003CF601C13DF62AC632F62BC633F62CC67D
:1068D00038F62DC639F6C6EC33F02EC632F62FC682
:1068E00033F6C6EC33F030C632F631C633F6C6ECBA
:1068F00033F02AC632F62BC633F62CC636F62DC632
:1069000037F6D6EC33F02EC632F62FC633F6D6EC79
:1069100033F030C632F631C633F6D6EC33F03851A8
:10692000365F3951D8A03929375F69EC37F036C660
:1069300000F137C601F175EC37F000C13EF601C138
:106940003FF63AC632F63BC633F63CC636F63DC68F
:1069500037F6D6EC33F03EC632F63FC633F6D6EC09
:1069600033F00794120018C100F119C101F11AC1E6
:1069700002F11BC103F1000E046F000E056F010E42
:10698000066F000E076F9FEC36F029A1DEEF34F0A2
:106990002051D8B4DEEF34F018C100F119C101F173
:1069A0001AC102F11BC103F1000E046F000E056F46
:1069B0000A0E066F000E076F9FEC36F01200010101
:1069C000045100130551011306510213075103131B
:1069D00012000101186B196B1A6B1B6B12002AC194
:1069E00082F40401300E822748EC0FF02BC182F4B0
:1069F0000401300E822748EC0FF02CC182F4040110
:106A0000300E822748EC0FF02DC182F40401300EC5
:106A1000822748EC0FF02EC182F40401300E822749
:106A200048EC0FF02FC182F40401300E822748ECAD
:106A30000FF030C182F40401300E822748EC0FF0D1
:106A400031C182F40401300E822748EC0FF032C1CC
:106A500082F40401300E822748EC0FF033C182F437
:106A60000401300E822748EC0FF012002FC182F48F
:106A70000401300E822748EC0FF030C182F404018B
:106A8000300E822748EC0FF031C182F40401300E41
:106A9000822748EC0FF032C182F40401300E8227C5
:106AA00048EC0FF033C182F40401300E822748EC29
:106AB0000FF01200060E1E6E060E1F6E060E206EE2
:106AC0001E2E60EF35F01F2E60EF35F0202E60EFA8
:106AD00035F08B84020E1E6E020E1F6E020E206EAB
:106AE0001E2E70EF35F01F2E70EF35F0202E70EF58
:106AF00035F08B9412000101005305E1015303E1CD
:106B0000025301E1002B3EEC36F069EC37F03951CD
:106B1000006F3A51016F420E046F4B0E056F000E6D
:106B2000066F000E076F7FEC36F000C104F101C163
:106B300005F102C106F103C107F118C100F119C145
:106B400001F11AC102F11BC103F107B2ACEF35F03C
:106B500073EC36F0AEEF35F06EEC36F000C118F1A4
:106B600001C119F102C11AF103C11BF1120069EC54
:106B700037F059C100F15AC101F1060EBDEC0BF01E
:106B8000E8CF04F1070EBDEC0BF0E8CF05F1080EDD
:106B9000BDEC0BF0E8CF06F1090EBDEC0BF0E8CF31
:106BA00007F16EEC36F000C124F101C125F102C1FC
:106BB00026F103C127F1290E046F000E056F000EA8
:106BC000066F000E076F7FEC36F0EE0E046F430E7B
:106BD000056F000E066F000E076F73EC36F024C1D0
:106BE00004F125C105F126C106F127C107F17FECAB
:106BF00036F000C11CF101C11DF102C11EF103C13B
:106C00001FF1120EBDEC0BF0E8CF04F1130EBDEC3A
:106C10000BF0E8CF05F1140EBDEC0BF0E8CF06F158
:106C2000150EBDEC0BF0E8CF07F10D0E006F000E56
:106C3000016F000E026F000E036F7FEC36F0180E2E
:106C4000046F000E056F000E066F000E076F9FECBD
:106C500036F01CC104F11DC105F11EC106F11FC1B2
:106C600007F173EC36F06A0E046F2A0E056F000E02
:106C7000066F000E076F6EEC36F01200BF0EFA6E54
:106C8000200E3A6F396BD89000370137023703373F
:106C9000D8B04FEF36F03A2F44EF36F039073A07C5
:106CA0000353D8B412000331070B80093F6F033937
:106CB0000F0B010F396F80EC5FF0406F390580ECEE
:106CC0005FF0405D405F396B3F33D8B039273933CF
:106CD0003FA964EF36F040513927120001018EECD4
:106CE00037F0D8B01200010103510719346F51EC8D
:106CF00037F0D8900751031934AF800F120001010B
:106D0000346B75EC37F0D8A08BEC37F0D8B01200AC
:106D100060EC37F069EC37F01F0E366FA1EC37F0FE
:106D20000B35D8B051EC37F0D8A00335D8B01200ED
:106D3000362F8EEF36F034B178EC37F012000101C7
:106D4000346B04510511061107110008D8A075EC29
:106D500037F0D8A08BEC37F0D8B01200086B096B75
:106D60000A6B0B6BA1EC37F01F0E366FA1EC37F0FE
:106D700007510B5DD8A4C9EF36F006510A5DD8A4BF
:106D8000C9EF36F00551095DD8A4C9EF36F00451BA
:106D9000085DD8A0DCEF36F00451085F0551D8A09B
:106DA000053D095F0651D8A0063D0A5F0751D8A0EE
:106DB000073D0B5FD8900081362FB6EF36F034B127
:106DC00078EC37F0346B75EC37F0D890A5EC37F0F1
:106DD00007510B5DD8A4F9EF36F006510A5DD8A42F
:106DE000F9EF36F00551095DD8A4F9EF36F00451FA
:106DF000085DD8A008EF37F0003F08EF37F0013FFB
:106E000008EF37F0023F08EF37F0032BD8B4120039
:106E100034B178EC37F012000101346B75EC37F0C7
:106E2000D8B01200AAEC37F0200E366F00370137C9
:106E30000237033711EE33F00A0E376FE7360A0ECA
:106E4000E75CD8B0E76EE552372F1EEF37F0362FEC
:106E500016EF37F034B12981D890120001010A0EE3
:106E6000346F200E366F11EE29F03451376F0A0E51
:106E7000D890E652D8B0E726E732372F39EF37F00F
:106E80000333023301330033362F33EF37F0E7504B
:106E9000FF0FD8A00335D8B0120029B178EC37F035
:106EA0001200045100270551D8B0053D01270651B5
:106EB000D8B0063D02270751D8B0073D032712007E
:106EC0000051086F0151096F02510A6F03510B6F96
:106ED00012000101006B016B026B036B12000101D8
:106EE000046B056B066B076B12000335D8A012000C
:106EF0000351800B001F011F021F031F003F88EF7B
:106F000037F0013F88EF37F0023F88EF37F0032B6F
:106F1000342B032512000735D8A012000751800B2F
:106F2000041F051F061F071F043F9EEF37F0053F94
:106F30009EEF37F0063F9EEF37F0072B342B0725E7
:106F400012000037013702370337083709370A378D
:106F50000B3712000101296B2A6B2B6B2C6B2D6BED
:106F60002E6B2F6B306B316B326B336B1200010168
:106F70002A510F0B2A6F2B510F0B2B6F2C510F0B1C
:106F80002C6F2D510F0B2D6F2E510F0B2E6F2F517C
:106F90000F0B2F6F30510F0B306F31510F0B316FC3
:106FA00032510F0B326F33510F0B336F1200899C2C
:106FB000000EC76E200EC66E9E96C69EC50EC96E8A
:106FC000FF0E9EB602D0E82EFCD79E96C69E000EFF
:106FD000C96EFF0E9EB602D0E82EFCD7C9CF00F6D0
:106FE0009E96C69E000EC96EFF0E9EB602D0E82E7B
:106FF000FCD7C9CF01F6898C1200000EC76E200E97
:10700000C66E899C9E96C69EC80EC96EFF0E9EB621
:1070100002D0E82EFCD79E96C69E000EC96EFF0ECB
:107020009EB602D0E82EFCD7C9CF02F69E96C69E29
:10703000000EC96EFF0E9EB602D0E82EFCD7C9CF57
:1070400003F69E96C69E000EC96EFF0E9EB602D037
:10705000E82EFCD7C9CF0AF69E96C69E000EC96ED2
:10706000FF0E9EB602D0E82EFCD7C9CF0BF69E9637
:10707000C69E000EC96EFF0E9EB602D0E82EFCD74B
:10708000C9CF12F69E96C69E000EC96EFF0E9EB622
:1070900002D0E82EFCD7C9CF13F6898C1200000E5F
:1070A000C76E200EC66E899C9E96C69EE80EC96E5F
:1070B000FF0E9EB602D0E82EFCD79E96C69E000E0E
:1070C000C96EFF0E9EB602D0E82EFCD7C9CF1AF6C5
:1070D0009E96C69E000EC96EFF0E9EB602D0E82E8A
:1070E000FCD7C9CF1BF69E96C69E000EC96EFF0E3A
:1070F0009EB602D0E82EFCD7C9CF22F69E96C69E39
:10710000000EC96EFF0E9EB602D0E82EFCD7C9CF86
:1071100023F69E96C69E000EC96EFF0E9EB602D046
:10712000E82EFCD7C9CF2AF69E96C69E000EC96EE1
:10713000FF0E9EB602D0E82EFCD7C9CF2BF6898C65
:107140001200000EC76E200EC66E899C9E96C69ECB
:10715000240EC96EFF0E9EB602D0E82EFCD79E9676
:10716000C69EE40EC96EFF0E9EB602D0E82EFCD776
:10717000898C899C9E96C69E200EC96EFF0E9EB677
:1071800002D0E82EFCD79E96C69E5F0EC96EFF0EFB
:107190009EB602D0E82EFCD7898C899C9E96C69E0E
:1071A000210EC96EFF0E9EB602D0E82EFCD79E9629
:1071B000C69EC00EC96EFF0E9EB602D0E82EFCD74A
:1071C000898C899C9E96C69E260EC96EFF0E9EB621
:1071D00002D0E82EFCD79E96C69E000EC96EFF0E0A
:1071E0009EB602D0E82EFCD7898C120010A806D0DB
:1071F0008994000EC76E220EC66E05D08984000EDB
:10720000C76E220EC66E050EE82EFED7120010A81D
:1072100002D0898401D08994050EE82EFED7120091
:10722000F6EC38F09E96C69E000EC96EFF0E9EB616
:1072300002D0E82EFCD79E96C69E000EC96EFF0EA9
:107240009EB602D0E82EFCD7C9CFAFF59E96C69E5B
:10725000000EC96EFF0E9EB602D0E82EFCD7C9CF35
:10726000B0F59E96C69E000EC96EFF0E9EB602D069
:10727000E82EFCD7C9CFB1F59E96C69E000EC96E0A
:10728000FF0E9EB602D0E82EFCD7C9CFB2F59E966F
:10729000C69E000EC96EFF0E9EB602D0E82EFCD729
:1072A000C9CFB3F59E96C69E000EC96EFF0E9EB660
:1072B00002D0E82EFCD7C9CFB4F59E96C69E000E2C
:1072C000C96EFF0E9EB602D0E82EFCD7C9CFB5F529
:1072D00007EC39F01200F6EC38F09E96C69E800E50
:1072E000C96EFF0E9EB602D0E82EFCD79E96C69EB3
:1072F000AFC5C9FFFF0E9EB602D0E82EFCD79E9602
:10730000C69EB0C5C9FFFF0E9EB602D0E82EFCD7C0
:107310009E96C69EB1C5C9FFFF0E9EB602D0E82E4E
:10732000FCD79E96C69EB2C5C9FFFF0E9EB602D080
:10733000E82EFCD79E96C69EB3C5C9FFFF0E9EB62B
:1073400002D0E82EFCD79E96C69EB4C5C9FFFF0E9C
:107350009EB602D0E82EFCD79E96C69EB5C5C9FF44
:10736000FF0E9EB602D0E82EFCD707EC39F01200D3
:10737000F6EC38F09E96C69E070EC96EFF0E9EB6BE
:1073800002D0E82EFCD79E96C69E000EC96EFF0E58
:107390009EB602D0E82EFCD7C9CFAFF59E96C69E0A
:1073A000000EC96EFF0E9EB602D0E82EFCD7C9CFE4
:1073B000B0F59E96C69E000EC96EFF0E9EB602D018
:1073C000E82EFCD7C9CFB1F59E96C69E000EC96EB9
:1073D000FF0E9EB602D0E82EFCD7C9CFB2F507EC5F
:1073E00039F0F6EC38F09E96C69E22C0C9FFFF0E1B
:1073F0009EB602D0E82EFCD79E96C69E000EC96EA1
:10740000FF0E9EB602D0E82EFCD7C9CFB6F507EC2A
:1074100039F01200F6EC38F09E96C69E870EC96EC3
:10742000FF0E9EB602D0E82EFCD79E96C69EAFC534
:10743000C9FFFF0E9EB602D0E82EFCD79E96C69ED0
:10744000B0C5C9FFFF0E9EB602D0E82EFCD79E96AF
:10745000C69EB1C5C9FFFF0E9EB602D0E82EFCD76E
:107460009E96C69EB2C5C9FFFF0E9EB602D0E82EFC
:10747000FCD707EC39F0F6EC38F09E96C69E23C098
:10748000C9FFFF0E9EB602D0E82EFCD79E96C69E80
:10749000B6C5C9FFFF0E9EB602D0E82EFCD707EC9A
:1074A00039F01200F6EC38F09E96C69E870EC96E33
:1074B000FF0E9EB602D0E82EFCD79E96C69E000E0A
:1074C000C96EFF0E9EB602D0E82EFCD79E96C69ED1
:1074D000800EC96EFF0E9EB602D0E82EFCD79E9697
:1074E000C69E800EC96EFF0E9EB602D0E82EFCD757
:1074F0009E96C69E800EC96EFF0E9EB602D0E82EE6
:10750000FCD707EC39F01200F6EC38F09E96C69ED8
:10751000870EC96EFF0E9EB602D0E82EFCD79E964F
:10752000C69E000EC96EFF0E9EB602D0E82EFCD796
:107530009E96C69E000EC96EFF0E9EB602D0E82E25
:10754000FCD79E96C69E800EC96EFF0E9EB602D0D8
:10755000E82EFCD79E96C69E800EC96EFF0E9EB684
:1075600002D0E82EFCD707EC39F0120010A82DD07D
:10757000F6EC38F09E96C69E23C0C9FFFF0E9EB65D
:1075800002D0E82EFCD79E96C69E450EC96EFF0E11
:107590009EB602D0E82EFCD707EC39F0F6EC38F0B6
:1075A0009E96C69E8F0EC96EFF0E9EB602D0E82E26
:1075B000FCD79E96C69E000EC96EFF0E9EB602D0E8
:1075C000E82EFCD707EC39F01200F6EC38F09E9666
:1075D000C69E23C0C9FFFF0E9EB602D0E82EFCD780
:1075E0009E96C69E010EC96EFF0E9EB602D0E82E74
:1075F000FCD707EC39F0F6EC38F09E96C69E910E5B
:10760000C96EFF0E9EB602D0E82EFCD79E96C69E8F
:10761000A50EC96EFF0E9EB602D0E82EFCD707EC71
:1076200039F01200F6EC38F09E96C69E23C0C9FFD2
:10763000FF0E9EB602D0E82EFCD79E96C69E810E07
:10764000C96EFF0E9EB602D0E82EFCD707EC39F0CB
:107650001200F6EC38F09E96C69E23C0C9FFFF0EBE
:107660009EB602D0E82EFCD79E96C69E010EC96E2D
:10767000FF0E9EB602D0E82EFCD707EC39F01200C0
:10768000F6EC38F09E96C69E910EC96EFF0E9EB621
:1076900002D0E82EFCD79E96C69EA50EC96EFF0EA0
:1076A0009EB602D0E82EFCD707EC39F01200F6ECBB
:1076B00038F09E96C69E910EC96EFF0E9EB602D001
:1076C000E82EFCD79E96C69E000EC96EFF0E9EB693
:1076D00002D0E82EFCD707EC39F012000501256B2B
:1076E000266B276B286B899A400EC76E200EC66EDC
:1076F0009E96C69E030EC96EFF0E9EB602D0E82E61
:10770000FCD79E96C69E27C5C9FFFF0E9EB602D027
:10771000E82EFCD79E96C69E26C5C9FFFF0E9EB6D4
:1077200002D0E82EFCD79E96C69E25C5C9FFFF0E47
:107730009EB602D0E82EFCD79E96C69EC952FF0E7A
:107740009EB602D0E82EFCD7898A0F01C950FF0AE5
:1077500001E1120005012E51130A05E005012E5129
:10776000170A0CE012000501E00E256FFF0E266FD0
:107770000F0E276F000E286FC7EF3BF00501E00EDC
:10778000256FFF0E266FFF0E276F000E286F899A58
:10779000400EC76E200EC66E9E96C69E030EC96E24
:1077A000FF0E9EB602D0E82EFCD79E96C69E27C539
:1077B000C9FFFF0E9EB602D0E82EFCD79E96C69E4D
:1077C00026C5C9FFFF0E9EB602D0E82EFCD79E96B6
:1077D000C69E25C5C9FFFF0E9EB602D0E82EFCD777
:1077E0009E96C69EC952FF0E9EB602D0E82EFCD7CA
:1077F000898A0F01C950FF0A1DE005012E51130AA5
:1078000005E005012E51170A0BE012000501000EDC
:10781000256F000E266F100E276F000E286F1200C6
:107820000501000E256F000E266F000E276F010E5A
:10783000286F12000501256B266B276B286B05014D
:107840002E51130A05E005012E51170A0CE0120013
:107850000501000E216F000E226F080E236F000E2F
:10786000246F3CEF3CF00501000E216F000E226FEB
:10787000800E236F000E246F21C500F122C501F197
:1078800023C502F124C503F125C504F126C505F180
:1078900027C506F128C507F1DFEC34F000C125F556
:1078A00001C126F502C127F503C128F5899A400ECA
:1078B000C76E200EC66E9E96C69E030EC96EFF0E44
:1078C0009EB602D0E82EFCD79E96C69E27C5C9FF5D
:1078D000FF0E9EB602D0E82EFCD79E96C69E26C509
:1078E000C9FFFF0E9EB602D0E82EFCD79E96C69E1C
:1078F00025C5C9FFFF0E9EB602D0E82EFCD79E9686
:10790000C69EC952FF0E9EB602D0E82EFCD7898AC9
:10791000C950FF0A08E104C125F505C126F506C1D5
:1079200027F507C128F5D8900501243323332233E6
:1079300021332151E00B216F2167A6EF3CF0226734
:10794000A6EF3CF02367A6EF3CF024673CEF3CF049
:107950000501200E2527E86A2623E86A2723E86A1E
:1079600028231200E86A05012E51130A06E00501DA
:107970002E51170A0BE0020E120005012851000AD1
:1079800003E12751F00B07E0010E12000501285119
:10799000000A01E0010E120029C500F12AC501F11B
:1079A0002BC502F12CC503F125C504F126C505F14F
:1079B00027C506F128C507F16EEC36F003BF1200AB
:1079C000B2EC3CF0D8A444EF3DF0899A400EC76E6B
:1079D000200EC66E9E96C69E060EC96EFF0E9EB601
:1079E00002D0E82EFCD7898A899A9E96C69E020EFE
:1079F000C96EFF0E9EB602D0E82EFCD79E96C69E9C
:107A000027C5C9FFFF0E9EB602D0E82EFCD79E9672
:107A1000C69E26C5C9FFFF0E9EB602D0E82EFCD733
:107A20009E96C69E25C5C9FFFF0E9EB602D0E82EC3
:107A3000FCD79E96C69E000EC96EFF0E9EB602D063
:107A4000E82EFCD7898A899A9E96C69E050EC96E35
:107A5000FF0E9EB602D0E82EFCD79E96C69EC95257
:107A6000FF0E9EB602D0E82EFCD7C9B02DEF3DF038
:107A7000898A0501200E2527E86A2623E86A27233C
:107A8000E86A2823CCEF3CF01200899A400EC76EBA
:107A9000200EC66E9E96C69E060EC96EFF0E9EB640
:107AA00002D0E82EFCD7898A899A9E96C69EC70E78
:107AB000C96EFF0E9EB602D0E82EFCD7898A05015A
:107AC000256B266B276B286B1200899A400EC76EB8
:107AD000200EC66E9E96C69E050EC96EFF0E9EB601
:107AE00002D0E82EFCD79E96C69EC952FF0E9EB6C7
:107AF00002D0E82EFCD7C9CF37F5898A1200899ABF
:107B0000400EC76E200EC66E9E96C69EB90EC96EFA
:107B1000FF0E9EB602D0E82EFCD7898A1200899A01
:107B2000400EC76E200EC66E9E96C69EAB0EC96EE8
:107B3000FF0E9EB602D0E82EFCD7898AFF0EE82EF3
:107B4000FED71200B2EC3CF0D8A41200899A400E85
:107B5000C76E200EC66E9E96C69E030EC96EFF0EA1
:107B60009EB602D0E82EFCD79E96C69E27C5C9FFBA
:107B7000FF0E9EB602D0E82EFCD79E96C69E26C566
:107B8000C9FFFF0E9EB602D0E82EFCD79E96C69E79
:107B900025C5C9FFFF0E9EB602D0E82EFCD79E96E3
:107BA000C69EC952FF0E9EB602D0E82EFCD7898A27
:107BB0000F01C950FF0AD8A499EF40F00501FE0E4D
:107BC000376F10EC39F0AFC538F5B0C539F5B1C530
:107BD0003AF5B2C53BF5B3C53CF5B4C53DF5B5C501
:107BE0003EF50784B6C166F1B7C167F1B8C168F167
:107BF000B9C169F14BC14FF14CC150F14DC151F1C7
:107C00004EC152F157C159F158C15AF185EC2AF0D1
:107C100000C13FF501C140F502C141F503C142F584
:107C2000050161671BEF3EF062671BEF3EF0636783
:107C30001BEF3EF064671FEF3EF02CEF3EF061C596
:107C400004F162C505F163C506F164C507F16EEC88
:107C500036F003BF99EF40F059C143F55AC144F5DE
:107C6000B9C545F5BAC546F5E6EC33F036C649F573
:107C700037C64AF50601406745EF3EF0416745EFDC
:107C80003EF0426745EF3EF0436749EF3EF05AEF62
:107C90003EF069EC37F06FEC37F036C600F137C6CE
:107CA00001F140C604F141C605F16EEC36F003AFB8
:107CB00099EF40F00101036B026B1AC600F11BC67D
:107CC00001F101AF68EF3EF0FF0E026FFF0E036F90
:107CD0000101076B066B1CC604F11DC605F105AF5B
:107CE00076EF3EF0FF0E066FFF0E076F73EC36F077
:107CF0000101076B066B1EC604F11FC605F105AF37
:107D000086EF3EF0FF0E066FFF0E076F73EC36F046
:107D10000101076B066B20C604F121C605F105AF12
:107D200096EF3EF0FF0E066FFF0E076F73EC36F016
:107D3000D89001010333023301330033D89001019D
:107D4000033302330133003300C14BF501C14CF55D
:107D50000101036B026B22C600F123C601F101AFE2
:107D6000B6EF3EF0FF0E026FFF0E036F0101076BCF
:107D7000066B24C604F125C605F105AFC4EF3EF03D
:107D8000FF0E066FFF0E076F73EC36F00101076BF5
:107D9000066B26C604F127C605F105AFD4EF3EF009
:107DA000FF0E066FFF0E076F73EC36F00101076BD5
:107DB000066B28C604F129C605F105AFE4EF3EF0D5
:107DC000FF0E066FFF0E076F73EC36F0D8900101BF
:107DD0000333023301330033D890010103330233FC
:107DE0000133003300C14DF501C14EF50101036BB4
:107DF000026B2AC600F12BC601F101AF04EF3FF080
:107E0000FF0E026FFF0E036F0101076B066B2CC69E
:107E100004F12DC605F105AF12EF3FF0FF0E066F1E
:107E2000FF0E076F73EC36F00101076B066B2EC671
:107E300004F12FC605F105AF22EF3FF0FF0E066FEC
:107E4000FF0E076F73EC36F00101076B066B30C64F
:107E500004F131C605F105AF32EF3FF0FF0E066FBA
:107E6000FF0E076F73EC36F0D89001010333023335
:107E700001330033D890010103330233013300335F
:107E800000C14FF501C150F50101036B026B02C641
:107E900000F103C601F101AF52EF3FF0FF0E026F98
:107EA000FF0E036F0101076B066B04C604F105C6E4
:107EB00005F105AF60EF3FF0FF0E066FFF0E076F95
:107EC00073EC36F00101076B066B06C604F107C6BA
:107ED00005F105AF70EF3FF0FF0E066FFF0E076F65
:107EE00073EC36F00101076B066B08C604F109C696
:107EF00005F105AF80EF3FF0FF0E066FFF0E076F35
:107F000073EC36F0D89001010333023301330033B0
:107F1000D8900101033302330133003300C151F51E
:107F200001C152F50101036B026B0AC600F10BC6D9
:107F300001F101AFA0EF3FF0FF0E026FFF0E036FE4
:107F40000101076B066B0CC604F10DC605F105AF08
:107F5000AEEF3FF0FF0E066FFF0E076F73EC36F0CB
:107F60000101076B066B0EC604F10FC605F105AFE4
:107F7000BEEF3FF0FF0E066FFF0E076F73EC36F09B
:107F80000101076B066B10C604F111C605F105AFC0
:107F9000CEEF3FF0FF0E066FFF0E076F73EC36F06B
:107FA000D89001010333023301330033D89001012B
:107FB000033302330133003300C153F501C154F5DB
:107FC0000101036B026B12C600F113C601F101AF90
:107FD000EEEF3FF0FF0E026FFF0E036F0101076B24
:107FE000066B14C604F115C605F105AFFCEF3FF0B2
:107FF000FF0E066FFF0E076F73EC36F00101076B83
:10800000066B16C604F117C605F105AF0CEF40F07C
:10801000FF0E066FFF0E076F73EC36F00101076B62
:10802000066B18C604F119C605F105AF1CEF40F048
:10803000FF0E066FFF0E076F73EC36F0D89001014C
:108040000333023301330033D89001010333023389
:108050000133003300C155F501C156F50794050100
:10806000210E326F899A400EC76E200EC66E9E9604
:10807000C69E060EC96EFF0E9EB602D0E82EFCD735
:10808000898A899A9E96C69E020EC96EFF0E9EB67A
:1080900002D0E82EFCD79E96C69E27C5C9FFFF0ECC
:1080A0009EB602D0E82EFCD79E96C69E26C5C9FF76
:1080B000FF0E9EB602D0E82EFCD79E96C69E25C522
:1080C000C9FFFF0E9EB602D0E82EFCD725EE37F092
:1080D000322F02D077EF40F09E96C69EDECFC9FFCA
:1080E000FF0E9EB602D0E82EFCD768EF40F0898ADA
:1080F000899A9E96C69E050EC96EFF0E9EB602D048
:10810000E82EFCD79E96C69EC952FF0E9EB602D0A0
:10811000E82EFCD7C9B082EF40F0898A0501200E15
:108120002527E86A2623E86A2723E86A28235AECE9
:1081300035F0120021C500F122C501F123C502F17D
:1081400024C503F1899A400EC76E200EC66E9E9616
:10815000C69E0B0EC96EFF0E9EB602D0E82EFCD74F
:108160009E96C69E02C1C9FFFF0E9EB602D0E82EA3
:10817000FCD79E96C69E01C1C9FFFF0E9EB602D0D7
:10818000E82EFCD79E96C69E00C1C9FFFF0E9EB684
:1081900002D0E82EFCD79E96C69EC952FF0E9EB610
:1081A00002D0E82EFCD725EE37F00501200E326F05
:1081B0009E96C69EC952FF0E9EB602D0E82EFCD7F0
:1081C000C9CFDEFF322FD8EF40F0898A1200899A9A
:1081D000400EC76E200EC66E9E96C69E900EC96E4D
:1081E000FF0E9EB602D0E82EFCD79E96C69E000ECD
:1081F000C96EFF0E9EB602D0E82EFCD79E96C69E94
:10820000000EC96EFF0E9EB602D0E82EFCD79E96D9
:10821000C69E000EC96EFF0E9EB602D0E82EFCD799
:108220009E96C69EC952FF0E9EB602D0E82EFCD77F
:10823000C9CF2DF59E96C69EC952FF0E9EB602D09E
:10824000E82EFCD7C9CF2EF5898A12005AEC35F0FA
:10825000B9C5E8FFD70802E35AEC35F0B9C5E8FF25
:10826000C80802E35AEC35F0B9C5E8FFB90802E3E3
:108270005AEC35F0B9C5E8FFAA0802E35AEC35F02C
:10828000B9C5E8FF9B0802E35AEC35F0B8EC39F0C9
:108290007FEC3DF0F29CF29E8B94C69AC290898C42
:1082A0009482948C720ED36ED3A4FED789968A9052
:1082B0009390FF0EE8CF00F0E82EFED7002EFCD7FB
:1082C0008150F294F29A9E909D909E929D92F29887
:0C82D000F292F290F286F28E0300FF00A2
:10BF0000E844F926000C160C2B0C3F0C520C640C68
:10BF1000760C860C960CA50CB30CC10CCF0CDC0C6B
:06BF2000E80CF40C000C1B
:00000001FF
